:040000000C94011249
:100004000C9400000C9400000C9400000C9400006C
:100014000C9400000C9400000C948A270C940000AB
:100024000C9400000C943B150C9400000C940000FC
:100034000C9400000C9400000C9400000C94DB144D
:100044000C9400000C9470260C9400000C948926E7
:100054000C9400000C9400000C9400000C9400001C
:100064000C9400000C9400000C9400000C9400000C
:100074000C9400000C94AE260C9400000C944927B8
:100084000C9400000C9400001000000102040810FD
:1000940020408000000040008000C00000014001BA
:1000A4000500C11100000300D90B00000300C111B9
:1000B4000300170E0300D90B00000500E008000040
:1000C4000A00C1110A00170E0A00D90B0A00C11157
:1000D4000A00170E2800D90B0000000000000000E1
:1000E400000000000000000000000000000000000C
:1000F40000000000000000000000070018C02020DD
:1001040020204D904D9040104010489047102020E2
:10011400202018C007000000000007001FC03FE0B7
:100124003FE0727072707FF07FF0777078F03FE09C
:100134003FE01FC007000000000007800F100E30D2
:100144000C7008F001F003F007F007F003F001F081
:1001540008F00C700E300F1007001E008F00C7004F
:10016400E300F100F800FC00FE00FE00FC00F800D3
:10017400F100E300C7008F001E007E0081008100B3
:10018400810081008100FF00810081008100FF0067
:1001940081008100810081007E00000000000200D7
:1001A400020007000F801FC03FE03FE03FE01AC09D
:1001B40007000F80000000000000000000000000A5
:1001C40000000000000006000F000F000600000001
:1001D40000000000000000000000FFF0FFF0FFF04E
:1001E400FFF0FFF0FFF0F9F0F0F0F0F0F9F0FFF0BD
:1001F400FFF0FFF0FFF0FFF0FFF000000000000050
:100204000000060009001080108010801080090092
:1002140006000000000000000000FFF0FFF0FFF007
:10022400FFF0F9F0F6F0EF70EF70EF70EF70F6F0AA
:10023400F9F0FFF0FFF0FFF0FFF000000000000015
:1002440001E000601EA03320618061806180330082
:100254001E000000000000000000000000000780F5
:100264000CC01860186018600CC0078003000300FD
:100274000FC003000300000000000200030003801D
:1002840003C002C002C00280020002000E001E0071
:100294001E000C000000000000000C000E000B000B
:1002A40009800CC00E400B4009C038C0784078402B
:1002B40031C003C003C0018000000000020002003E
:1002C40027201FC018C030607070306018C01FC075
:1002D40027200200020000000000000000001000BF
:1002E40018001C001E001F001F801F001E001C00A1
:1002F4001800100000000000000000000000008052
:100304000180038007800F801F800F800780038097
:1003140001800080000000000000000002000700CF
:100324000F801FC0020002000200020002001FC072
:100334000F800700020000000000000019801980EF
:1003440019801980198019801980198019801980E1
:100354000000198019800000000000001FE036C072
:1003640066C066C066C036C01EC006C006C006C0F1
:1003740006C006C006C00000000000001F8030C098
:10038400300030001F8030C030C01F8000C000C06B
:1003940030C01F80000000000000000000000000CA
:1003A4000000000000000000000000000000000049
:1003B4001FE01FE01FE000000000020007000F80A4
:1003C4001FC00200020002000200020002001FC05F
:1003D4000F80070002001FC0000000000200070099
:1003E4000F801FC00200020002000200020002008F
:1003F40002000200020000000000000002000200EF
:1004040002000200020002000200020002001FC0FB
:100414000F80070002000000000000000000000040
:1004240000000100018001C03FE001C00180010023
:1004340000000000000000000000000000000000B8
:10044400000004000C001C003FE01C000C00040031
:100454000000000000000000000000000000000098
:1004640000000000000000000000400040004000C8
:10047400400040007FE00000000000000000000099
:100484000000088018C038E07FF038E018C0088009
:100494000000000000000000000000000000000058
:1004A40000000000020007000F801FC03FE07FF043
:1004B4000000000000000000000000000000000038
:1004C400000000007FF03FE01FC00F800700020023
:1004D4000000000000000000000000000000000018
:1004E4000000000000000000000000000000000008
:1004F40000000000000000000000060006000F00DD
:100504000F000F000F000F00060006000600000099
:100514000000060006000000000000000000198032
:1005240019801980198000000000000000000000FC
:1005340000000000000000000000000006600660EB
:1005440006603FF00CC00CC0198019807FC03300D6
:1005540033003300000000000000060006001F8086
:100564003FC0360036003F801FC006C006C03FC0F3
:100574001F800600060000000000000000000010BC
:100584003830387038E001C0038007000E001C00CA
:1005940038E070E060E000000000000007000D801B
:1005A400198019801B000E001E003E00336033C00A
:1005B40031803BC01E60000000000E000E000E00E3
:1005C400060006000C00000000000000000000000F
:1005D40000000000000000000000038006000E0080
:1005E4000C001C001C001C001C001C001C000C0047
:1005F4000E0006000380000000001C000600070037
:1006040003000380038003800380038003800300CE
:10061400070006001C0000000000000000000000AD
:1006240036C036C01F800F003FC00F001F8036C089
:1006340036C00000000000000000000000000000C0
:1006440000000600060006003FC03FC0060006008A
:100654000600000000000000000000000000000090
:100664000000000000000000000000000000000086
:100674000E000E000E0006000C000000000000003A
:1006840000000000000000003FC03FC00000000068
:100694000000000000000000000000000000000056
:1006A4000000000000000000000000000000000046
:1006B4000E000E000E0000000000000000100030CC
:1006C400007000E001C0038007000E001C00380029
:1006D400700060000000000000000F803FE0306008
:1006E400607060F061B0633066306C3078307030C8
:1006F40030603FE00F8000000000030007001F008F
:100704001F000300030003000300030003000300B1
:1007140003001FE01FE0000000001FC03FE07070F6
:100724006030607000E001C0038007000E001C0010
:1007340038007FF07FF0000000001FC03FE07070C1
:100744006030003000700FE00FC000600030603097
:1007540070703FE01FC00000000001C003C007C06C
:100764000EC01CC038C070C060C07FF07FF000C0F5
:1007740000C000C000C0000000007FF07FF06000F7
:10078400600060007FC03FE00070003000306030E7
:1007940070703FE01FC00000000003C007C00E00DF
:1007A4001C00380030007FC07FE070706030603023
:1007B40070703FE01FC0000000007FF07FF0006019
:1007C400006000C000C00180018003000300060037
:1007D40006000C000C00000000000F801FC038E071
:1007E4003060306038E01FC03FE0707060306030CF
:1007F40070703FE01FC0000000001FC03FE0707039
:100804006030603070703FF01FF0006000E001C0A5
:1008140003801F001E000000000000000000000014
:1008240000000E000E000E000000000000000E008C
:100834000E000E0000000000000000000000000098
:1008440000000E000E000E000000000000000E006C
:100854000E000E00060006000C0000C001C003805C
:1008640007000E001C00380038001C000E000700B2
:10087400038001C000C00000000000000000000070
:10088400000000003FE03FE0000000003FE03FE0E8
:1008940000000000000000000000300038001C00D0
:1008A4000E000700038001C001C0038007000E0092
:1008B4001C0038003000000000001F803FC070E0C2
:1008C400606060E001C003800700060006000600C7
:1008D400000006000600000000001FC03FE030607A
:1008E40067B06FB06DB06DB06DB06DB06FE067C0E4
:1008F40070003FC00FC000000000060006000F009B
:100904000F000F0019801980198030C03FC03FC00C
:10091400606060606060000000007F007F8061C0F4
:1009240060C060C061C07F807FC060E06060606064
:1009340060E07FC07F80000000000F801FC038E0AF
:100944003060600060006000600060006000306043
:1009540038E01FC00F80000000007F007F8061C06E
:1009640060C060606060606060606060606060C0C3
:1009740061C07F807F00000000007FE07FE06000B6
:100984006000600060007F807F8060006000600025
:1009940060007FE07FE0000000007FE07FE0600017
:1009A4006000600060007F807F8060006000600005
:1009B400600060006000000000000FC01FE03860AD
:1009C40030006000600063E063E06060606030609D
:1009D40038601FE00FE0000000006060606060604D
:1009E4006060606060607FE07FE0606060606060C5
:1009F400606060606060000000001F801F8006006F
:100A040006000600060006000600060006000600B2
:100A140006001F801F80000000000060006000606E
:100A24000060006000600060006000606060606002
:100A340070C03FC01F8000000000606060E061C0C3
:100A4400638067006E007C007C006E00670063803A
:100A540061C060E060600000000060006000600051
:100A64006000600060006000600060006000600082
:100A740060007FE07FE000000000606070E070E0F4
:100A840079E079E06F606F60666066606060606006
:100A940060606060606000000000606070607060B2
:100AA40078606C606C60666066606360636061E07F
:100AB40060E060E06060000000000F001F8039C04B
:100AC40030C060606060606060606060606030C0C2
:100AD40039C01F800F00000000007F807FC060E0ED
:100AE40060606060606060E07FC07F806000600084
:100AF400600060006000000000000F001F8039C02B
:100B040030C060606060606060606060636033C07B
:100B140039C01FE00F60000000007F807FC060E0EC
:100B240060606060606060E07FC07F8067006380B9
:100B340061C060E06060000000001F803FC070E0A2
:100B44006060600070003F801FC000E00060606073
:100B540070E03FC01F80000000003FC03FC006009F
:100B64000600060006000600060006000600060051
:100B7400060006000600000000006060606060601F
:100B84006060606060606060606060606060606061
:100B940030C03FC01F800000000060606060606083
:100BA40030C030C030C01980198019800F000F0088
:100BB4000F000600060000000000606060606060D6
:100BC4006060606060606060666066606F6079E06D
:100BD40070E070E06060000000006060606030C041
:100BE40030C019800F00060006000F00198030C0C5
:100BF40030C060606060000000006060606030C011
:100C040030C0198019800F000F000600060006008E
:100C1400060006000600000000007FE07FE000C040
:100C240000C001800300060006000C00180030001C
:100C340030007FE07FE000000000666066600F0027
:100C44000F000F0019801980198030C03FC03FC0C9
:100C5400606060606060000000006F605FA039C089
:100C640030C060606060606060606060606030C020
:100C740039C01F800F000000000060606060000049
:100C84006060606060606060606060606060606060
:100C940030C03FC01F80000000001F801F8018006C
:100CA4001800180018001800180018001800180080
:100CB40018001F801F8000000000000000000000DA
:100CC4000000000000000000000000000000000020
:100CD4000000000000007FF07FF000000700070024
:100CE40007000600060003000000000000000000EA
:100CF40000000000000000000000000000000000F0
:100D0400000000001FC03FE000601FE03FE06060A3
:100D140060607FE03FE00000000060006000600071
:100D2400600060006F807FC070E060606060606041
:100D340060E07FC07F800000000000000000000031
:100D4400000000001F803FC0706060006000600011
:100D540070603FC01F800000000000600060006001
:100D6400006000601F603FE071E060606060606090
:100D740070603FE01FE00000000000000000000081
:100D8400000000001F803FC070607FE07FC06000F3
:100D940070003FC01F800000000007800F801C000F
:100DA4001800180018007F007F00180018001800B1
:100DB40018001800180000000000000000000000E7
:100DC400000000001FE03FE07060606070E03FE002
:100DD4001F60006000E03FC03F8060006000600072
:100DE400600060006F007F8071C060C060C060C040
:100DF40060C060C060C00000000000000000060089
:100E0400060000000E000E000600060006000600A4
:100E140006001F801F800000000000000000018009
:100E24000180000003800380018001800180018033
:100E34000180018019801F800F00300030003000D5
:100E4400300030003180338037003E003E003700F0
:100E5400338031C030C0000000000E000E000600D8
:100E6400060006000600060006000600060006004E
:100E740006001F801F80000000000000000000002A
:100E84000000000059807FC07FE066606660666095
:100E940066606660666000000000000000000000FC
:100EA400000000003F803FC030E0306030603060C0
:100EB400306030603060000000000000000000007E
:100EC400000000001F803FC070E0606060606060F0
:100ED40070E03FC01F800000000000000000000020
:100EE400000000007F807FC060E06060606070E0B0
:100EF4007FC06F80600060006000000000000000A0
:100F0400000000001FE03FE070606060606070E01F
:100F14003FE01F600060006000600000000000000F
:100F24000000000037C03FE038603000300030007F
:100F3400300030003000000000000000000000001D
:100F4400000000003F007F8060007F003F80018040
:100F540001807F803F00000000000000180018009E
:100F6400180018007F007F001800180018001800EF
:100F740018001F800F800000000000000000000027
:100F840000000000606060606060606060606060DD
:100F940070E03FE01F60000000000000000000005F
:100FA400000000006060606030C030C019801980AB
:100FB4000F000F0006000000000000000000000009
:100FC40000000000666066606660666066606F6070
:100FD4003FC039C010800000000000000000000085
:100FE4000000000060C071C03B801F000E001F00A5
:100FF4003B8071C060C000000000000000000000E1
:101004000000000030C030C0198019800F000F00AC
:10101400060006000C000C00180000000000000090
:10102400000000007FC07F80030006000C00180051
:1010340030007FC07FC0000000000000000060603E
:10104400000000001FC03FE000601FE03FE0606060
:1010540060607FE03FE0000000000000000060608E
:10106400000000001F803FC070E06060606060604E
:1010740070E03FC01F8000000000000000006060BE
:1010840000000000606060606060606060606060DC
:1010940070E03FE01F600000000000003F007F8020
:1010A40060C060C061C0678067C060E0606060600D
:1010B40060E067C0678000000000000000000000DE
:1010C400000006000F00198030C0606060607FE09F
:1010D4007FE000000000000000000F801FC038E027
:1010E400306060606000600060006000306038E084
:1010F4001FC00F8006001E001E00000000001980A3
:1011040019800000606060606060606060606060C2
:1011140070E03FE01F600000000000000180030059
:10112400060000001F803FC070607FE07FE0600029
:1011340070003FC01F8000000000000006000F0088
:10114400198000001FC03FE000601FE03FE06060C6
:1011540060607FE03FE000000000000000001980B4
:10116400198000001FC03FE000601FE03FE06060A6
:1011740060607FE03FE00000000000000C0006001B
:10118400030000001FC03FE000601FE03FE060601C
:1011940060607FE03FE000000000000006000900FE
:1011A400060000001FC03FE000601FE03FE06060F9
:1011B40060607FE03FE000000000000000000000ED
:1011C400000000001F803FC070E06000600060000D
:1011D40070E03FC01F8006001E00000006000F00E4
:1011E400198000001F803FC070607FE07FE06000D6
:1011F40060003FC01F800000000000000000198054
:10120400198000001F803FC070607FE07FE06000B5
:1012140060003FC01F800000000000000C000600BA
:10122400030000001F803FC070607FE07FE060002B
:1012340060003FC01F8000000000000000001B0091
:101244001B0000000E000E0006000600060006004B
:1012540006001F801F8000000000000006000F0031
:10126400198000000E000E000600060006000600AD
:1012740006001F801F800000000000000C00060014
:10128400030000000E000E00060006000600060023
:1012940006001F801F8000000000198019800000D4
:1012A400060006000F000F001980198030C03FC0EF
:1012B4007FE0606060600000000006000900060036
:1012C400000006000F000F001980198030C03FC0D5
:1012D4007FE06060606000000000018003000600A1
:1012E4007FE07FE0600060007F807F8060006000BE
:1012F40060007FE07FE000000000000000000000CC
:101304000000000000003DC0666006603FC066004B
:10131400660066603BC00000000007E007E00F00C5
:101324000F001F001B001BC033C033003F007F00B1
:10133400630063E063E000000000000006000F00AB
:10134400198000001F803FC070E0606060606060D2
:1013540070E03FC01F800000000000000000198002
:10136400198000001F803FC070E0606060606060B2
:1013740070E03FC01F800000000000000C00060069
:10138400030000001F803FC070E060606060606028
:1013940070E03FC01F8000000000000006000F0046
:1013A4001980000060606060606060606060606020
:1013B40070E03FE01F600000000000000C00060029
:1013C4000300000060606060606060606060606096
:1013D40070E03FE01F600000000000000000198082
:1013E4001980000030C030C0198019800F000F0030
:1013F400060006000C000C0018001980198000007B
:101404001F803FC070E0606060606060606060602A
:1014140070E03FC01F800000000000000000198041
:10142400198000006060606060606060606060609F
:1014340070E03FE01F6000000000000000000000BA
:10144400000000001F603FC071E0636066606C6074
:1014540078E03FC06F8000000000000000000780BB
:101464000FC00CC00C000C001F000C000C00180076
:101474003FE03BC0000000000000000000001F60CF
:101484003FC071E063606360666066606C606C605E
:1014940078E03FC06F800000000000000000000002
:1014A400000030C019800F0006000F00198030C002
:1014B40000000000000000000000038007C006C018
:1014C40006000600060006001F800600060006004F
:1014D400060036003E001C00000000000300060069
:1014E4000C0000001FC03FE000601FE03FE06060B0
:1014F40060607FE03FE000000000000003000600A1
:101504000C0000000E000E00060006000600060097
:1015140006001F801F80000000000000030006007A
:101524000C0000001F803FC070E06060606060607D
:1015340070E03FC01F8000000000000003000600B0
:101544000C0000006060606060606060606060600B
:1015540070E03FE01F6000000000000000000EC0CB
:101564001B8000003F803FC030E03060306030605E
:10157400306030603060000000000EC01B8000004E
:101584006060706078607C606E60676063E061E0FA
:1015940060E060606060000000001FC03FE0006029
:1015A4003FE07FE060607FE03FE000003FC03FC07D
:1015B400000000000000000000001F803FC070E039
:1015C4006060606070E03FC01F8000003FC03FC0AB
:1015D40000000000000000000000060006000000FB
:1015E4000600060006000E001C00380070606060F3
:1015F40070E03FC01F8000000000000000001FC01A
:101604003FE070706F306DB06F306DB06DB0707062
:101614003FE01FC0000000000000000000000000C8
:10162400FFE0FFE000600060006000600060000018
:101634000000000000000000000000000000300076
:10164400700030C031807B0006000DC0186030C0CF
:10165400018001E0000000000000000000003000F4
:10166400700030C031807B0006000D601B6033E0E9
:10167400006000600000000000000600060000009A
:1016840000000600060006000F000F000F000F0008
:101694000F0006000600000000000000000000002B
:1016A4000000000018C031806300318018C00000C1
:1016B4000000000000000000000000000000000026
:1016C400000000006300318018C031806300000016
:1016D40000000000000000000000888022208880B4
:1016E40022208880222088802220888022208880CE
:1016F400222088802220888022205550AAA055507C
:10170400AAA05550AAA05550AAA05550AAA0555019
:10171400AAA05550AAA05550AAA07770DDD0777022
:10172400DDD07770DDD07770DDD07770DDD0777065
:10173400DDD07770DDD07770DDD0060006000600BE
:101744000600060006000600060006000600060065
:101754000600060006000600060006000600060055
:101764000600060006000600FE00FE000600060055
:1017740006000600060006000600030006000C0032
:10178400060006000F000F001980198030C03FC00A
:101794007FE0606060600000000006000F001980B8
:1017A400060006000F000F001980198030C03FC0EA
:1017B4007FE060606060000000000C000600030031
:1017C400060006000F000F001980198030C03FC0CA
:1017D4007FE06060606000000000000000001FC047
:1017E4003FE0707067306DB06C306DB06730707012
:1017F4003FE01FC000000000000036003600360045
:10180400360036003600F600F6000600F600F60054
:101814003600360036003600360036003600360014
:101824003600360036003600360036003600360004
:101834003600360036003600360000000000000096
:10184400000000000000FE00FE000600F600F600A6
:1018540036003600360036003600360036003600D4
:10186400360036003600F600F6000600FE00FE00E4
:101874000000000000000000000000000600060058
:101884000F801FC03EC03600360036003EC01FC069
:101894000F8006000600000000006060606030C039
:1018A40030C0198019800F000F0006003FC00600E9
:1018B4003FC0060006000000000000000000000019
:1018C4000000000000000000FE00FE00060006000C
:1018D40006000600060006000600060006000600D4
:1018E400060006000600060007F007F000000000EE
:1018F40000000000000000000000060006000600D2
:101904000600060006000600FFF0FFF000000000DD
:1019140000000000000000000000000000000000C3
:101924000000000000000000FFF0FFF006000600C9
:101934000600060006000600060006000600060073
:10194400060006000600060007F007F00600060081
:101954000600060006000600060000000000000065
:101964000000000000000000FFF0FFF00000000095
:101974000000000000000000000006000600060051
:101984000600060006000600FFF0FFF00600060051
:1019940006000600060006000600000000000EC057
:1019A4001B8000001FC03FE000601FE03FE060605C
:1019B40060607FE03FE0000000000EC01B8000007C
:1019C400060006000F000F001980198030C03FC0C8
:1019D4007FE0606060600000000036003600360082
:1019E40036003600360037F037F030003FF03FF075
:1019F40000000000000000000000000000000000E3
:101A04000000000000003FF03FF0300037F037F0F6
:101A14003600360036003600360036003600360012
:101A2400360036003600F7F0F7F00000FFF0FFF064
:101A340000000000000000000000000000000000A2
:101A4400000000000000FFF0FFF00000F7F0F7F0E6
:101A540036003600360036003600360036003600D2
:101A640036003600360037F037F0300037F037F004
:101A74003600360036003600360000000000000054
:101A8400000000000000FFF0FFF00000FFF0FFF096
:101A940000000000000000000000360036003600A0
:101AA400360036003600F7F0F7F00000F7F0F7F0F4
:101AB40036003600360036003600000060606F6085
:101AC4003FC070E0606060606060606070E03FC074
:101AD4006F606060000000000000000000000F0064
:101AE4001F80188018001C000E0007000F8019804A
:101AF40019801F800F00000000003F003F8031C0AC
:101B040030C030603060786078603060306030C001
:101B140031C03F803F000000000006000F00198024
:101B24007FE07FE0600060007F807F806000600075
:101B340060007FE07FE00000000019801980000051
:101B44007FE07FE0600060007F807F806000600055
:101B540060007FE07FE00000000018000C00060039
:101B64007FE07FE0600060007F807F806000600035
:101B740060007FE07FE00000000000000600060037
:101B84000600060006000600000000000000000039
:101B940000000000000000000000018003000600B7
:101BA4001F801F80060006000600060006000600CF
:101BB40006001F801F800000000006000F0019802F
:101BC4001F801F80060006000600060006000600AF
:101BD40006001F801F80000000001980198000008B
:101BE4001F801F800600060006000600060006008F
:101BF40006001F801F80000000000600060006008B
:101C04000600060006000600FE00FE0000000000BC
:101C140000000000000000000000000000000000C0
:101C2400000000000000000007F007F006000600B6
:101C340006000600060006000600FFF0FFF0FFF0B5
:101C4400FFF0FFF0FFF0FFF0FFF0FFF0FFF0FFF018
:101C5400FFF0FFF0FFF0FFF0FFF0000000000000D5
:101C640000000000000000000000FFF0FFF0FFF0A3
:101C7400FFF0FFF0FFF0FFF0FFF0060006000600A3
:101C84000600060006000000060006000600060026
:101C94000600060006000000000018000C00060004
:101CA4001F801F80060006000600060006000600CE
:101CB40006001F801F8000000000FFF0FFF0FFF00F
:101CC400FFF0FFF0FFF0FFF0FFF000000000000065
:101CD4000000000000000000000001800300060076
:101CE4001F803FC070E06060606060606060606042
:101CF40070E03FC01F8000000000000000000000F2
:101D040000000F00198030C030C03F8031C030C0A7
:101D140030C031C03F803000300006000F00198011
:101D24001F803FC070E06060606060606060606001
:101D340070E03FC01F800000000018000C00060087
:101D44001F803FC070E060606060606060606060E1
:101D540070E03FC01F8000000000000000001D80F4
:101D6400370000001F803FC070E06060606060600A
:101D740070E03FC01F80000000000EC01B80000008
:101D84001F803FC070E060606060606060606060A1
:101D940070E03FC01F800000000000000000000051
:101DA400000060C060C060C060C060C071C07FC01F
:101DB4007EC06000600060006000000000003C0025
:101DC4003C0018001F801FC018C018C01FC01F800F
:101DD40018003C003C00000000003C003C001800DF
:101DE4001F801FC018C018C018C018C01FC01F8093
:101DF40018003C003C0000000000018003000600C5
:101E040060606060606060606060606060606060CE
:101E140030C03FC01F800000000006000F00198082
:101E240060606060606060606060606060606060AE
:101E340030C03FC01F800000000018000C000600E6
:101E4400606060606060606060606060606060608E
:101E540030C03FC01F80000000000000000001806F
:101E64000300060030C030C0198019800F000F0035
:101E7400060006000C000C00180001800300060098
:101E8400606030C019800F000600060006000600DE
:101E940006000600060000000000000000000780A5
:101EA40007800000000000000000000000000000A7
:101EB40000000000000000000000030006000C0009
:101EC400000000000000000000000000000000000E
:101ED40000000000000000000000000000000000FE
:101EE4000000000000001F801F80000000000000B0
:101EF40000000000000000000000000000000000DE
:101F04000000060006001F801F8006000600000077
:101F14001F801F800000000000000000000000007F
:101F24000000000000001F801F8000001F801F8031
:101F3400000000000000000000000000000070002D
:101F4400180030C01980730006000D601B6033E078
:101F54000060006000000000000000001FE036C0C8
:101F640066C066C066C036C01EC006C006C006C0D5
:101F740006C006C006C00000000000001F8030C07C
:101F8400300030001F8030C030C01F8000C000C04F
:101F940030C01F80000000000000000000000000AE
:101FA40000000600060000003FC03FC0000006001D
:101FB4000600000000000000000000000000000017
:101FC40000000000000013000F00000000000000EB
:101FD400000000000000000000000F001F801980B6
:101FE40019801F800F0000000000000000000000A6
:101FF40000000000000000000000000000000000DD
:10200400000000000000108039C039C010800000BA
:1020140000000000000000000000000000000000BC
:10202400000000000000020007000700020000009A
:102034000000000000000000000018003800180034
:10204400180018000000000000000000000000005C
:10205400000000000000000000003C0006001C001E
:1020640006003C000000000000000000000000002A
:10207400000000000000000000003C0006001C00FE
:1020840030003E00000000000000000000000000DE
:10209400000000000000000000000000000000003C
:1020A40000000F000F000F000F000F000F000000D2
:1020B400000000000000000000000000000000001C
:1020C400000000000000000000000000000000000C
:1020D4000000000000000000000000001E00600777
:1020E4007E0700F01EF060F77EF7FBDE1F00E007BE
:1020F400FF0700F81FF8E0FFFFFF00001E00600765
:102104007E0700F01EF060F77EF7FBDE1F00E0079D
:10211400FF0700F81FF8E0FFFFFF03004A00530029
:102124004A00A3004A00030072007B00720003000F
:10213400EA0003009A0053009A000300EA0000003A
:1021440040008000C00000014001A00050000000D9
:102154000000A000A000500000000000F8000000F3
:10216400FF000000FF0000007F80001E0F80007F42
:10217400E7C0007FFFE0003FFFE00007FFC0000171
:10218400FFC00001FF800001FF0003FFFE0007FF06
:10219400FC0007FFF00003FFF00003FFFE00001F38
:1021A400FFC001FFFFF001FFFFF801FFFFF8007F10
:1021B400FFF80007FE00003FFF00007FFF80007F64
:1021C400FF80007FC100001FE000001FF000001F1F
:1021D400F000000FE0000007C0000007C000000787
:1021E400C00000078000000300000003000000029C
:1021F400000000000000000000000000E0000000FB
:1022040000000003900000000000000E1800000011
:102214000000003808000000000000C018000000A2
:10222400000003807000000000000C01C0000001E9
:102234008006300700000003C00F401C00000006A9
:10224400E01DC0700000000C3039C1C0000000184F
:102254001871C7180000001C0CE1DC7C0000000EA3
:1022640007C3F1C40000000703860706000000034B
:10227400800E1C0200000001C01C3003000000009E
:10228400E03818010080000070700FC183C00000A6
:1022940038E003E08E6006001DC00020FC200F0023
:1022A4000F8000307030198007000010003030C0FB
:1022B4000000001800E06060000000080380603047
:1022C4000000000C0E003018000000043800180C48
:1022D40000000006E0000C06000000038000060376
:1022E40000000000000003018000000000000180E5
:1022F400C0000000000000C0C0000000000000603A
:10230400C000000000000030C000000000000030E9
:10231400C000000000000030C000000000000030D9
:10232400C000000000000030C000000000000030C9
:10233400C000000000000030C000000000000030B9
:10234400C000000000000030C000000000000030A9
:10235400E0000000000000307000000000000030C9
:1023640018000000000000300C00000000000030E5
:10237400040000000000003FFC0000000000003FDB
:10238400FC00436F6C6F72546F7563682056732042
:10239400312E32382000426C6F636B200043616C35
:1023A4006962726174696F6E004F4B002530325858
:1023B4000025303458002533642E2530326400253E
:1023C40035640025640025326400253364004444E8
:1023D4000000256400253032580025313064004F58
:1023E4004E00426C6F636B0077616C6C610001009E
:1023F4002D4E414E00000100D90BF2230000F89449
:10240400EE27ECBBF1E0F5BFE5BFE0936C00F8E12B
:10241400F1BDE1BD8DE0A2E0BB27ED938A95E9F71C
:1024240080E090E1A0E0B1E0ED930197E9F7EAEFF5
:10243400F3E285919591009761F0A591B59105908E
:102444001590BF01F00105900D920197E1F7FB0192
:10245400F0CFEFEFEDBFE0E1EEBFC0E0D3E00C94CE
:10246400AF15E881E03019F01C9A1D9A02C01C983F
:102474001D983CC00E94EA2C0E94EA2C0E94EF2C7A
:10248400FA93EA93EFE3F0E00E94F42C08950E949B
:10249400072A0E94652A0E94FA2C0E94EA2C0E94B4
:1024A400002D0E94171AE6E8F3E20E94052DE09140
:1024B4000B03E05DEA930E940F1A0E94EA2C0E942B
:1024C400092D0E94171AEAE9F3E20E94052D0E94E1
:1024D4000E2DEA930E94EB160895E881E064E7B9B3
:1024E400369A349BFECF349AE4B1F5B1219608951F
:1024F400E881F981AA81BB81AE17BF071CF4EA1BEE
:10250400FB0B06C0A881B981EA81FB81EA1BFB0BA6
:102514002496089528970E943635EFE0E0936100F1
:10252400E1E00E94132DE5E00E941A2D0E94212D66
:10253400E0939106F0939206E0919D06F0919E0639
:10254400E0938F06F0939006E1E0EA93C6DFE09310
:102554009D06F0939E06EFE0E0936100E8E00E94A0
:10256400132DEAE00E941A2D0E94262DE0938D0679
:10257400F0938E06E0919B06F0919C06E0938B0607
:10258400F0938C06E0E0EA93A8DFE0939B06F093D7
:102594009C060E94262DA0918D06B0918E06EA0F0E
:1025A400FB1FA0919B06B0919C060E942B2D8F01CE
:1025B4000E94212DA0919106B0919206EA0FFB1F73
:1025C400A0919D06B0919E060E942B2D9F01E09143
:1025D4008D06F0918E060E94322DFF93EF930E9498
:1025E400262D0E94322DAF91BF91EA0FFB1FFF935E
:1025F400EF93E0919B06F0919C060E94322DAF91DF
:10260400BF91EA0FFB1FE0939706F0939806E091C1
:102614009106F09192060E94382DFF93EF930E9449
:10262400212D0E94382DAF91BF91EA0FFB1FFF931C
:10263400EF93E0919D06F0919E060E94382DAF9194
:10264400BF91EA0FFB1FE0939906F0939A06A091BD
:102654009706B0919806E4E1F0E00E94A9320E2EAC
:10266400A0919906B0919A06E4E1F0E00E94A932A3
:10267400E02919F00E944219B9C0009393061093FF
:10268400940620939506309396060E943E2DA63418
:10269400E0E0BE0724F4A7E8B6E00E94432D0E94C0
:1026A400492D989724F40E944E2D98970CF010C051
:1026B4000E943E2D1A9721F4E1E0F0E00E94532D90
:1026C4000E943E2D989721F4E2E0F0E00E94532D01
:1026D4000E94492D999724F00E944E2D99970CF44D
:1026E40085C0A1E8B6E00E94432D0E94582D0E94A7
:1026F400492D0E945D2D0E94642D0E94692DE0EFFA
:10270400F0E060E070E00E94DC327F936F93FF930F
:10271400EF930E946E2D0F010E94582DDF01F001EE
:10272400EA1BFB0BAF91BF918F919F910E94A43242
:102734000E942C330E94642D0E94732D0E944E2D02
:102744000E945D2DEC83FD836E837F83AC81BD810C
:102754008E819F81E0E4F1E060E070E00E94DC3271
:102764007F936F93FF93EF930E94782D0F010E9444
:10277400732DDF01F001EA1BFB0BAF91BF918F9129
:102784009F910E94A4320E942C33EC83FD836E83BC
:102794007F83E0910503E03049F4E885F985E0930F
:1027A4007506F0937606EC81FD810EC0EC81FD8107
:1027B400E0937506F09376060E94692DEFEEF0E043
:1027C40060E070E00E948532E0937706F09378062B
:1027D400E0917506F0917606FA93EA93E091770614
:1027E400F0917806FA93EA930E94B2180E943D355C
:1027F4000C94E9160E943E1AE2E0E09301030E9461
:102804007D2D0E947D2D0E94321AE1EAF3E20E949E
:10281400052DE4E1EA930E948B16E0E9F1E00E94C1
:10282400822DE4E1EA930E948B160E94862D0E9479
:10283400303514F4A895F9CFE2E0E09300030E9448
:10284400EA2C0E948B2D0E94321AEBE10E94902DFB
:102854000E94862D5F9714F4A895FACF0E94972DB5
:10286400A0E0B0E00E94A02DEAE5F0E00E94A32DD4
:102874000E94582D0E94A72D0E94862D5E9714F069
:10288400A895FACF0E94EA2C0E948B2D0E94AB2DB2
:10289400E2E0E09300030E94B22D0E94321AEAE1C2
:1028A4000E94902D0E94862D5F9714F4A895FACF6C
:1028B4000E94972DA2E0B0E00E94A02DE2E8F0E093
:1028C4000E94A32D0E946E2D0E94A72D0E94862D8A
:1028D4005E9714F0A895FACF0E94B22D0E94AB2DFA
:1028E4000E94B72D0E94EA2C0E94321AE8E10E944D
:1028F400902D0E94862D5F9714F4A895FACF0E941C
:10290400BF2DA4E0B0E00E94A02DEAEAF0E00E940E
:10291400A32D0E94732D0E94A72D0E94862D5E97E1
:1029240014F0A895FACFE9E6F0E0FA93EA930E944E
:10293400EA2C0E94AB2D0E94B72DEEE1F1E00E943B
:10294400A32DE9E10E94902D0E94862D5F9714F437
:10295400A895FACF0E94BF2DA6E0B0E00E94A02D5A
:10296400E2EDF0E00E94A32D0E94782D0E94A72D95
:102974000E94862D5E9714F0A895FACFE9E6F0E060
:10298400FA93EA93EEE1F1E0FA93EA930E94AB2D15
:102994000E947D2DEAEFF0E00E94A32DEDEAF3E220
:1029A4000E94052DE0EDF7E00E94822D0E943E1A60
:1029B40008950E94C82DE2EBE2BF78940E946F183C
:1029C400A9DDA0912208A13028F0E0912208E1506D
:1029D400E0932208E0912108E0932008E6B3AFEFEA
:1029E400EA27E0932108E03019F0E3E0E0932308BC
:1029F400E0912108A0912008EA17A9F4A0912108E8
:102A0400A03021F0A0912208A03069F0A091210803
:102A1400A03041F4A0912208A03021F4A091230811
:102A2400A03009F40FC0F894E091FF06E160E09350
:102A3400FF067894E2E3E0932208E0912308E15052
:102A4400E0932308AEE1B8E00E94432DE091FE0339
:102A5400EF5FE093FE03A091FE03AE3149F4A09131
:102A6400FD03E3E8EA27E093FD03E0E0E093FE03DF
:102A740008C00E94C82D1A93E3E8E4BD0E94982977
:102A84001991E991EFBFF991E991B991A9919991BE
:102A9400899179916991F9901990099018951A93EF
:102AA400A895BED1E13011F00C949615E091E7069B
:102AB400E1501E2FA091E606A13021F40E94D62DEC
:102AC400E03009F412C00E94D62DE093FC06E1E048
:102AD400E093FF060E94DD2DBF010E94DD2DE08101
:102AE400E260DB01EC930E94E32DA091E606A230A4
:102AF40011F0A430C9F40E94D62DE093FD06E5E15F
:102B0400E093FC06E1E0E093FF060E94D62DE0305E
:102B140029F00E94DD2DE081E27009F405C01A93CA
:102B2400E2E0EA930E949F1AE091FD03E07889F0C5
:102B3400E091FD03EF77E093FD030E94411DE091D6
:102B4400FD03E07131F0E091FD03E270EA930E942D
:102B540077190E949D2719910895E0E0E5BFE0935D
:102B64006D00E0936C00EBBBEFEFEABBE0E0E8BB89
:102B7400E7BBE5BBEFEFE4BBE0EFE2BBE1BBE0E3C7
:102B8400E3B9ECEBE2B9E0E0E0936200E0936100CA
:102B9400EFE0E0936500E0936400E0E0E0BFE7E08D
:102BA400E3BFE2EBE2BFE0E0E1BFEFBDEEBDEDBDB0
:102BB400ECBDE7BDE6BDEBBDEABDE9BDE8BDE09314
:102BC4007900E0937800E3E0E5BDE3E8E2BFE0E00C
:102BD400E3BDE0938B00EAE0E0938A00E0E0E09359
:102BE4008900E0938800E0938100E0938000E2E1B3
:102BF400E0938700E4E3E0938600E0E0E09385005F
:102C0400E0938400E0938300E0938200E0936A0001
:102C1400E0E3EABFE0E4E9BFE8BFE1E4E7BFE0E006
:102C2400E0937D00EBB9E8EDEAB9E6E0E0939500C6
:102C3400E0E0E0939000E3E3E9B9E0E0E0939B0097
:102C4400E8EDE0939A00E6E0E0939D00E0E0E09395
:102C54009800E9E1E0939900E0E8E8B9E0E0E0BD3C
:102C6400E0E4E7B9E7E8E6B9E0B5EF7EE0BDE0E12E
:102C7400E0937000E0E0E0937200E4E4E093740019
:102C8400EEE1E1BDEEE0E1BD78940E94D22527D3C8
:102C9400E1E0EA930E9433120E940E2DE53128F000
:102CA400A8E0B0E0E4E10E949F330E94491221E0D1
:102CB4000E94582D0F010E946E2D0E161F0644F41B
:102CC4000E94732D0F010E94782D0E161F060CF022
:102CD40091DDE1E0EA931DD000E010E00436E0E08D
:102CE4001E0724F40E949D27E03009F005C00E94CD
:102CF400E82D0F5F1F4FF2CF0436E0E01E0734F0DB
:102D04000E94862D5F9714F00E94FC13C8DEFECF4C
:102D1400FFCFE881E03021F4EAEAF0E00E94EB2DF5
:102D2400A881A13021F4E4EAF0E00E94EB2DA8810F
:102D3400A23021F4E0EBF0E00E94EB2DA881A33057
:102D440021F4EEEBF0E00E94EB2DA881A43021F4F5
:102D5400E4ECF0E00E94EB2D66C31A9310E00E94AD
:102D6400F02DE03031F00E94F02DEA9356D31F5F2E
:102D7400F6CF1881239608951A930A93E0E0E0931E
:102D84009F06E093A00610E0143190F400E00330B5
:102D940068F4A3E01A9FF001EA55F94FDF01EE272A
:102DA400A00FBE1FE0E2EC930F5FF1CF1F5FECCFEB
:102DB400D4C12A970E94F72DE3ECF3E2FA93EA9345
:102DC400EE85FF850E94A4320E94FB2DC6DF2C965F
:102DD40008952A970E94F72DEAECF3E2FA93EA9316
:102DE400EE85FF27662777270E94FB2DB6DF2B96FB
:102DF40008951A930A9300E010E00E94022EE03036
:102E040021F00832E0E01E070CF007C00E94022EF9
:102E1400EA9303D30F5F1F4FF0CF198108812AC3B0
:102E2400E091E506A091E406EA17C1F00E94092E9C
:102E3400AE0FBF1FEC91E093E7060E94092EEA0F44
:102E4400FB1FE181E093E606A091E506AF5FEAE0AF
:102E54000E943133E093E506E1E00895E0E008954F
:102E64000E94112EA981A0830E94112E3196A8815F
:102E7400A083A091E406AF5FEAE00E943133E093BF
:102E8400E406C9C21A930E941B2EE45FFC4FA0E023
:102E9400A0830E941B2EEA5EFC4F108117FF05C021
:102EA400E12F0E94202EA0E0A08316FF05C0E12F91
:102EB4000E94272EA0E0A0830E941B2EEA5EFC4FF6
:102EC400A0E0A0830E941B2EEB5EFC4FA0E0A08339
:102ED4001881A1C2AD970E943435EAADFBADAEAD09
:102EE400BFADEA0FFB1FAF0110E0143188F50E945B
:102EF400D62DE03041F10E942E2EDF010E9467336F
:102F0400DF01ECADFDADEA17FB07E9F40E94342EB6
:102F1400DF01EEADFFADAE17BF07ACF00E94342E5B
:102F24004E175F0784F00E943D2EAE0FBF1FEEAD1B
:102F3400FFADAE17BF073CF00E943D2EAE0FBF1F82
:102F44004A175B070CF402C01A939CDF1F5FCDCFB6
:102F540010E0143110F00C9469180E94D62DE03062
:102F640011F00C946718ACE01A9FF001E45FFC4F79
:102F7400AFA90E944C2EE35FFC4FAEADBFADA08362
:102F8400B1830E942E2EACADBDADA083B183ACE065
:102F94001A9FF001EF5EFC4FAAAD0E944C2EEE5E2C
:102FA400FC4FA8AD0E944C2EED5EFC4FA091020395
:102FB4000E944C2EEC5EFC4FA0910303A0830E9460
:102FC400DD2D0F01E091FC03E295E07FA091040365
:102FD400EA0FD001EC930E94512EA0E00E944C2EE7
:102FE400E95EFC4FA0E0A083E0E0EE83EDA9FEA93A
:102FF400309741F00E94572EEFA9F8ADFA93EA9367
:103004000E94952AEBA9FCA9309731F00E94572E13
:10301400EDA9FEA90E945C2EE0E0EEA70E94572EC7
:103024000E94A02A3E2F3B30A8F000E00E94602EB0
:1030340011F00C3008F002C00F5FF8CF0E94602E30
:1030440049F40E94682E30E00E94512EDF01E02FE7
:10305400E058EC93E0E0E88B3130F0F000E00E94BF
:10306400722E11F00C3008F002C00F5FF8CF0E94EE
:10307400722E91F4ABE00A9FF001EB5FFB4FFA93E1
:10308400EA93FE0138960E945C2E30E00E94512E95
:10309400DF01E02FE05CEC933130A8F000E00E9407
:1030A400602E11F00C3008F002C00F5FF8CF0E94C0
:1030B400602E49F40E94682E30E00E94512EDF01F8
:1030C400E02FE058EC93E12F03C01F5F42CFEFEFF6
:1030D4000E943B35EF96219608951A930A930E9415
:1030E4007A2E3097D1F1E0917B06F0917C063097EF
:1030F40069F50E947A2E0E947133E0937B06F09367
:103104007C06309731F4E0E0F0E00E94EB2DE0E043
:103114001AC00E947F2E0E947A2E0E947133F59568
:10312400E7958F01D801E0E0F1E00E940233E093DB
:103134008700D801E0E0F1E00E943433E093860098
:103144000E947F2EE0E4E0938B0007C0ABE7B6E07B
:10315400ED91FD913197FE93EE93099119910895A4
:103164001A930A9300E010E0143110F00C94F8184C
:103174000E94D62DE030C1F10E94342EAC81BD8175
:10318400EA17FB0764F50E942E2EDF010E946733C5
:10319400AA81BB81EA17FB0714F5ACE01A9FF00182
:1031A400E35FFC4F608171811A9FF001EF5EFC4F79
:1031B4000E94872EAC81BD81AE17BF0784F40E94A4
:1031C4002E2E60817181ACE01A9FF001EE5EFC4FFF
:1031D4000E94872EAA81BB81AE17BF070CF004C0E2
:1031E400E12FEF5F0E2F02C01F5FBECF003081F0D2
:1031F400E0918506F0918606A02FB0E0EA17FB0760
:1032040031F0A0918506B0918606109709F401C0AB
:103214002BC00E943E2D159791F40A93E1E0EA93A6
:103224001FDEE02FF0E0E0938506F0938606E02FA2
:10323400F0E00E948C2EE3E0F0E00E94532D0E9407
:103244003E2D5E9721F4E4E0F0E00E94532DA0911E
:103254007906B0917A06139734F0E5E0F0E0E09354
:103264008306F093840608C00E94912E0E94532D79
:10327400E0E0F0E00E948C2E1981088126960895E2
:10328400E0918506F09186063097A1F00E943E2DCC
:10329400999734F4E0918506EA93E2E0EA93E0DD5D
:1032A4000E943E2DDD9734F0E0918506EA93E4E038
:1032B400EA93D6DDE0E0F0E00E94532D0E94912EC7
:1032C400E0938506F0938606E0E0F0E00E948C2E01
:1032D400E0E0F0E0E0938106F09382060895CCD01C
:1032E4004BDDE5E1E093FC0608950E943435A0919E
:1032F400A106A43120F4A091A206A33008F032C0A4
:10330400E091A1060E94982E8F01E091A206F0E0C0
:10331400A4E1B0E00E94D7329F010E949E2EECE00F
:10332400F0E0FA93EA930E94A32E0E9496320E9440
:10333400F42CEE81E030B1F0E091A106A3E0EA9F25
:10334400F001EA55F94FDF01E091A206F0E0AE0F7B
:10335400BF1F4C9155270E949E2E4A93E0E0EA93AA
:103364000E9461260E943B35279608950E94EF2C07
:10337400A0910703B0910803AE17BF075CF4E09176
:103384000104F0910204A0910903B0910A03AE175D
:10339400BF070CF040C0E0910703F0910803FA93D3
:1033A400EA93E0910903F0910A030E94A72E0E9478
:1033B4006126A0917D06B0917E06549734F4A091C5
:1033C4007F06B091800613970CF012C0E0917D0641
:1033D400F0917E06A3E0B0E00E94AF32EA55F94FC7
:1033E400A0917F06B0918006EA0FFB1FA981A083FC
:1033F4000E94AE2EA0910703B09108030E94B42E40
:103404000E94B82EE0917D06F0917E063196E093FD
:103414007D06F0937E0622960895E881EA93E09172
:103424000303EA93A3DF21960895EA81FB81E093E5
:103434007D06F0937E06E881F981E0937F06F093A0
:103444008006AA81BB81ECE0F0E00E94D7320E94A2
:10345400B82EA881B981E4E1F0E00E94D73206C019
:10346400EA81FB810E94B82EE881F981E093090387
:10347400F0930A03249608950E94BD2E143120F47B
:103484001A9300DD1F5FFACF0E94EA2C0E94EA2CF7
:103494000E94EF2CFA93EA93E0910104F091020464
:1034A4000E94F42C10E01C3048F4A9E21A9FF001A9
:1034B400E757FB4FA0E0A0831F5FF5CF10E01C305F
:1034C40048F4ABE01A9FF001EB5FFB4FA0E0A08350
:1034D4001F5FF5CFE091FD03EF7EE093FD03E5C2AE
:1034E4000E94BD2E1431C0F40E942E2E0E94C52EBF
:1034F400AE17BF0764F00E942E2E0E94CC2EEA174E
:10350400FB072CF00E94512EE081E03009F402C048
:103514001A93B8DC1F5FE6CF0E94EA2CED81FE818E
:10352400FA93EA930E94EF2CFA93EA93A985BA8559
:103534000E94D32E0E94F42C9FC2EE970E94343531
:103544000E94D82EE03009F460C20E94D82EEFAF5A
:10355400E07851F00E94572EFE01EF5BFF4FE081AF
:103564000E94202E0E945C2EEFADE07451F00E9468
:10357400572EFE01EF5BFF4FE0810E94272E0E9431
:103584005C2E0E94572E0E94A02AEEAFE091000309
:10359400E9AFE0910103E8AF0E94FA2C0E94E32E08
:1035A400E35FFC4F008111810E94E32EE15FFC4F39
:1035B400208131810E94E32EEF5EFC4F408155272C
:1035C4000E94E32EEE5EFC4FE081F0E0DE01AE5B94
:1035D400BF4FED93FC930E94E32EED5EFC4FE08120
:1035E400EAAF0E94EB2EDF010E94A32E0E94D73285
:1035F4000E94F02E0E949E2E5A934A930E94F62E09
:10360400FA93EA93FE01EE5BFF4FE081EA930E9496
:1036140009260E949E2E0E94FD2E3A932A930E9410
:10362400032F0E94072F0E94122F0E94152F0E9421
:10363400E32EEB5EFC4FE081E07181F00E949E2E50
:103644005A934A930E94002D0E941B2FFA01E00F07
:10365400F11F35970E941F2F0E94242F0E94E32EF2
:10366400EB5EFC4FE081E07269F00E94072F369711
:103674000E942C2F0E94002D0E941B2F0E949E2E20
:103684000E94242F0E949E2E1A930A930E94152FA3
:103694000E94FD2E3A932A930E94FD2E0E94152F1C
:1036A4000E94312FA130B1F41A930A93F901319693
:1036B4000E94122FF9013196FA93EA930E94032F84
:1036C400F80131960E941F2FF8013196FA93EA937C
:1036D4000E94152F0E94312FA230E1F40E94072F7F
:1036E40031970E94122F0E94F62EE20FF31F31979A
:1036F400FA93EA930E94032FFA01E00FF11F319726
:103704000E941F2FFA01E00FF11F3197FA93EA93F9
:103714000E94152FFE01EC5BFF4FE081E03011F4B5
:103724000C94DB1C0E94E32EEC5EFC4FE081EAAFBC
:103734000E94AE2E0E94362F0E940233EBAFAEAD34
:10374400EA1710F40C94F71BE1E0E0930103E03076
:1037540041F00E94EB2EEE0FFF1F34960E94392F8A
:103764000CF009C0E2E0E09301030E94EB2EEE0F9F
:10377400FF1F0E94F02EDE01A05CBF4F0D90BC9194
:10378400A02D0E94432FEA1BFB0BDF010E944A2F4E
:103794000E944F2F32F4FE01E05CFF4F002401929F
:1037A4000082AEAD0E94562F0E94362F0E945E2FDB
:1037B400ECAF0E94312FA13021F40E94612F0E94AE
:1037C400662F0E94312FA23021F40E94612F0E94A3
:1037D4006E2FE0E0EFAF0E94742FE03029F00E94DA
:1037E400742F0E947C2FF7CFE4C0FE01E05CFF4FF2
:1037F4000190F081E02DEE0FFF1FDE01AE5BBF4FA5
:103804000D90BC91A02DAE1BBF0BE3E0F0E00E9435
:1038140002330E944F2F22F4E1E0F0E00E94F02EE8
:10382400EBADA2E0EA9FF001AEADAE17A8F5E1E082
:10383400E0930103E03041F00E94EB2E0E949A32A3
:1038440036960E94392F0CF009C0E2E0E0930103A0
:103854000E94EB2EEE0FFF1F0E94F02EEEADEDAF97
:10386400EDADE150EDAFEDAD0E94852FA03219F022
:10387400ADADA13008F404C0EDADE150EDAFF3CF30
:10388400ADAD0E94562FAE2FFA01B0E0EA17FB0748
:103894003CF3EDADE03011F4EBADEDAFADADECE0EC
:1038A400EA9FF0010E94362F0E945E2FECAF0E9427
:1038B400312FA13021F40E94612F0E94662F0E94B3
:1038C400312FA23021F40E94612F0E946E2FE0E07C
:1038D400EFAFEFAD0E94852FA03021F0EDADAFAD7D
:1038E400AE1708F005C00E94742F0E947C2FF1CF00
:1038F400EFAD0E94852FA03221F4EEADAFADAE172F
:1039040008F007C0EFADEF5FEFAFEDADEF5FEDAFE8
:10391400EFCFADADEEADEA1BAE2FEBADEA1778F00D
:10392400ADADEEADEA1BACE0EA9FF001A09100035F
:10393400EA9FF0010E94362F0E945E2F01C0E0E052
:10394400ECAF0E94312FA13081F40E94612F319697
:10395400FA93EA930E94EB2E3197DF010E94A32E83
:103964000E948C2F31960E94A32D0E94312FA230E9
:1039740071F40E94612FFA93EA930E94EB2E31971F
:10398400DF010E94A32E0E948C2F0E94A32DEFAD75
:103994000E94852FA03039F0ADADEFADEA1BAE2FFC
:1039A400EBADEA1708F405C00E94742F0E947C2F27
:1039B400EECF0E94E32EE95EFC4FE081E030F9F0A7
:1039C4000E94FA2C0E949E2E4BDDE0E0E09303035C
:1039D4000E94E32EE95EFC4FE081EA3040F00E9451
:1039E400E32EE95EFC4FE081EA93F3D908C00E941C
:1039F400E32EE95EFC4FE081E05DEA930EDDE9AD84
:103A0400E0930003E8ADE09301030E943B35EF9699
:103A1400279608951A9310E0E89422F8143148F494
:103A24000E94D62DE03011F00E94E32D1F5FA8956F
:103A3400F5CFE0E0E093030338C01A9310E01431AB
:103A4400C0F40E94D62DE03071F00E942E2E0E9408
:103A5400C52EEA17FB073CF40E942E2E0E94CC2EA2
:103A6400AE17BF070CF002C00E94E32D1F5FA8959C
:103A7400E6CFE0E0E09303031881259608951A93B6
:103A840010E0143190F40E94D62DE03029F00E9409
:103A9400DD2DE081E17009F406C01A93E091FD0385
:103AA400E170EA934ADD1F5FECCF199108952C97DA
:103AB4000E943435AD89BE890E944A2FED8BFE8B5E
:103AC400AB89BC890E944A2FEB8BFC8BED89FE8964
:103AD400A98DBA8DEA0FFB1FE98FFA8FEB89FC8958
:103AE400AF89B88DEA0FFB1FEF8BF88FED89FE8944
:103AF400AD89BE890E94972FEE87FF87688B798BEB
:103B0400EB89FC89AB89BC890E94972FAE85BF8560
:103B1400888999890E94E734EA87FB876C877D87C7
:103B240000E010E0EB89FC89E017F10714F40C9431
:103B3400E21DF8010E94A4320E941634EE83FF8332
:103B440068877987AE81BF81888599850E94993479
:103B5400AA85BB858C859D850E949934AE85BF85D9
:103B6400888999890E947A330E9449340E94DF33FC
:103B7400AF015A934A930E94CB2C2E2F33270E94D5
:103B84009E2FE98DFA8DE01BF10B0E94A52FED8D80
:103B9400FE8DE01BF10B0E94AF2F0E949E2FF801B7
:103BA400A98DBA8DEA0FFB1F0E94A52FF801AD8DD8
:103BB400BE8DEA0FFB1F0E94AF2F0F5F1F4FB2CFC6
:103BC4000E943B356B960895EA81F0E0EBBBF5BBB0
:103BD400F7E1F09365001F98E6E1E0936500F09348
:103BE4006500E881F981EBBBF5BBFFE1F09365006B
:103BF400EEE1E0936500F09365001F9A0C94D021E8
:103C0400E2E2EBBBE0E0E5BB0C94D6210C94E121AD
:103C14000E94B52FEFE1E0936500E4E6F0E00E9436
:103C2400822DE5EEEA93E0E0F0E80E94BB2FE0E0AD
:103C34000E94BF2FE1E0EA93E0E0F1E00E94BB2F95
:103C4400E2E0EA93E0E0F4E00E94BB2F0E94C32F7D
:103C54000E94C82FB9DFE8E0EA93E2E0F2E00E94B4
:103C6400BB2FE9E0EA930E94EA2C0E94E61DEAE0F9
:103C7400EA930E94EA2C0E94E61DECE0EA930E947B
:103C8400EA2C0E94E61DEDE0EA930E94EA2C0E94D1
:103C9400E61DEFE0EA930E94EA2C0E94E61DE0E1B3
:103CA400EA930E94EA2C0E94E61DE1E1EA930E9455
:103CB400092D0E94E61DE2E1EA930E94EA2C0E948B
:103CC400E61DE3E1EA930E94EA2C0E94E61D0E94AD
:103CD4007D2D0E947532E0E1EA93E0EBFBE10E9466
:103CE400BB2FE1E1EA930E94092D0E94E61D0E9488
:103CF4007D2D0E947532E2E1EA93EEE1F1E00E944B
:103D0400BB2F0E947D2D0E947532E3E1EA93E0E02F
:103D1400FFE10E94BB2FE9E2EA93EFE1F0E00E94A9
:103D2400BB2F0E947D2D0E947532E0E2EA930E942F
:103D3400EA2C0E94E61DE1E2EA930E94EA2C0E942A
:103D4400E61DA0910B03A13029F4EBE2EA93ECE029
:103D5400F0E004C0EBE2EA93E0E2F0E0FA93EA93E5
:103D64000E94E61DE0E3EA930E94EA2C0E94E61D0D
:103D7400E1E3EA930E94EA2C0E94E61DE2E3EA935F
:103D84000E94EA2C0E94E61DE5E3EA930E94EA2CD5
:103D94000E94E61DE6E3EA93E1E0F1E00E94BB2F16
:103DA400E7E30E94CB2FE8E30E94CB2FE9E30E94D4
:103DB400CB2FECE30E94CB2FEDE30E94CB2FE0E569
:103DC400EA930E94EA2C0E94CF2FE2E5EA930E9434
:103DD400EA2C0E94D62FA0910B03A13029F4E0E62F
:103DE400EA93E0E0F7EA04C0E0E6EA93E0E0F7E211
:103DF400FA93EA930E94E61DE1E60E94BF2FEAE6E9
:103E0400EA930E94EA2C0E94E61DE0E8EA930E94ED
:103E1400EA2C0E94E61DE1E8EA930E94EA2C0E9443
:103E2400E61DE2E8EA930E94EA2C0E94E61DE3E81C
:103E3400EA930E94EA2C0E94E61DE4E8EA930E94B9
:103E4400EA2C0E94E61DE5E8EA930E94EA2C0E940F
:103E5400E61DE0E9EA93E0E1F0E00E94BB2FE2E92D
:103E6400EA93E0E0F7E00E94BB2FE3E9EA930E94C3
:103E7400092D0E94E61DE5E9EA93EFE3F3E00E94D1
:103E8400BB2FE7E9EA930E94EA2C0E94E61DE8E9C9
:103E9400EA930E94EA2C0E94E61DE7E00E94BF2FED
:103EA4000E947D2D0E947532E7E0EA93E1E2F0E0A2
:103EB4000E94BB2FE7E0EA93E3E2F0E00E94BB2F0D
:103EC4000E947D2D0E947532E7E0EA93E3E7F1E07A
:103ED4000E94BB2F08950E94DD2FAE85AA2362F0B5
:103EE400AD85BE85A03FE0E0BE0734F4AB85BC855C
:103EF400AF33E1E0BE070CF04EC00E94EB2FAE0FD3
:103F0400BF1FA03FE0E0BE0714F00E94F02F0E9404
:103F1400F92FAE0FBF1FA034E1E0BE0714F00E94DA
:103F2400FE2F4985E0E50E940730E1E50E940B3051
:103F34000E941130E2E50E941430E3E50E9418303B
:103F44000E941130E0E20E940730E1E20E94143046
:103F540057DE0BBB15BB2EE13FE100E010E00E94F1
:103F64001E3064F050E0451730F020936500309324
:103F740065005F5FF8CF0F5F1F4FF1CF47DEE0E5CD
:103F8400EA930E94EA2C0E94CF2FE2E5EA930E9472
:103F9400EA2C0E94D62F52C00E94DD2F0E94EB2FE4
:103FA400EA17FB0729F50E94233014F40E942A30F3
:103FB400E3E0EA93E8E3F0E10E94BB2FE0E20E9431
:103FC4000730E1E20E9414301BDE0BBB15BB2EE16F
:103FD4003FE10B851C850E941E303CF02093650058
:103FE400309365000F5F1F4FF6CF0E94C32F24C08C
:103FF4000E94F92FEA17FB0729F50E943B3014F4BD
:104004000E942A30E0E20E940730E1E20E9414306C
:104014000E94021E0BBB15BB2EE13FE10D851E85E0
:10402400E985FA85E017F1073CF0209365003093A9
:1040340065000F5F1F4FF4CF0E94081E0E943B359E
:104044002F9608950E9442300E944930FF93EF93C7
:104054000E944D300E944930AF91BF91EA17FB078F
:10406400D8F10E942330ECF420E030E00E9450307C
:10407400E217F307ACF00E9442300E9457300E94CE
:1040840050300E945C30E1E2EA93EC85FD85E21B4E
:10409400F30B0E94BB2F0E9466302F5F3F4FE6CF89
:1040A40019C020E030E00E944D30E217F30794F08D
:1040B4000E9442300E9457300E944D300E945C3072
:1040C400E1E20E946C300E9411300E9466302F5F42
:1040D4003F4FE9CF0C94C4240E9442300E944930DF
:1040E400FF93EF930E944D300E944930AF91BF91EE
:1040F400EA17FB07E8F50E943B30ECF420E030E0DF
:104104000E947130E217F307ACF00E944D300E9418
:1041140057300E9471300E947830EE85FF85E21B93
:10412400F30B0E94BB2F0E947F300E9466302F5FEA
:104134003F4FE6CF1BC020E030E00E944230E21740
:10414400F307A4F00E944D300E9457300E94423081
:104154000E947830F901AE85BF850E9411300E941B
:104164007F300E9466302F5F3F4FE7CF0C94C4240A
:104174000C94C42425970E943435EB850E94853025
:104184000E949130103110F00C94362100E0E0913F
:1041940001030E1710F00C942E21E1E20E94073067
:1041A400E0E0EA87AA85A23010F00C9426210E9450
:1041B4009D30E252FF4F2491203011F40C942121C0
:1041C40027FF34C00E94AF30E2E2EBBBE0E0E5BB86
:1041D400E7E1E09365001F98F6E1F0936500E09352
:1041E4006500EE81EBBBEF81E5BBEFE1FEE1E0931F
:1041F4006500F0936500E093650031FF04C0F0931F
:104204006500E093650026FF10C0F0936500E0931D
:10421400650031FF06C0F0936500E09365004F5FD1
:104224005F4F220F4F5F5F4FEECF1F9A220F31FF78
:1042340002C04F5F5F4F4F5F5F4F0C94DE20EA85F3
:10424400EF5FEA870C94D420ED85FE853196ED87E7
:10425400FE870F5F0C94C920E885F9853296E887BC
:10426400F9871F5F0C94C4200E94C32F0C94CE25A1
:1042740023970E943435E9850E94853030910003EC
:1042840010E0EA851E1710F00C94B22100E0E091D2
:1042940001030E1710F00C94AF21E1E2EA93ED85CF
:1042A400FE850E94BB2FE0E0E887EB85A885AE176A
:1042B40010F00C94A7210E94B530203011F40C9416
:1042C400A22127FF34C00E94AF30E2E2EBBBE0E062
:1042D400E5BBE7E1E09365001F98F6E1F093650024
:1042E400E0936500EE81EBBBEF81E5BBEFE1FEE11E
:1042F400E0936500F0936500E093650031FF04C02E
:10430400F0936500E093650026FF10C0F09365000C
:10431400E093650031FF06C0F0936500E09365000B
:104324004F5F5F4F220F4F5F5F4FEECF1F9A220FF9
:1043340031FF02C04F5F5F4F4F5F5F4F0C945F21AF
:10434400E885EF5FE8870C945721EC85FD8531966D
:10435400EC87FD870F5F0C9449211F5F0C94432168
:104364000E94C32F0C94CE25EA81F0E0E5BBFBBB91
:10437400F7E1F09365001F98E6E1E0936500F093A0
:104384006500E881F981E5BBFBBBFFE1F0936500C3
:10439400EEE1E0936500F09365001F9A239608957B
:1043A400E2E2E5BBE0E0EBBBE7E1E09365001F98E8
:1043B400E6E1E0936500E7E1E093650008951F9A64
:1043C40008950E94B52FEFE1E0936500E8ECF0E07A
:1043D4000E94822DE6E4EA93E4EAF0E00E94CA3007
:1043E400E7E4EA93E3E5F0E00E94CA30E8E4EA9304
:1043F4000E94EA2CB9DFE9E4EA93E4E4F0E00E94E5
:10440400CA30EAE40E94CE30EBE4EA93E7E6F0E057
:104414000E94CA30ECE4EA93E3E3F0E00E94CA307D
:10442400EDE4EA93E7E7F0E00E94CA30EEE4EA93B1
:10443400E2E1F0E00E94CA30EFE4EA93ECE4F0E059
:104444000E94CA30E0E5EA93E6E4F0E00E94CA3054
:10445400E1E5EA93E4E4F0E00E94CA30E1E0EA93A3
:104464000E94002D0E94B6210E94D230E3E2EA931A
:10447400E5E9F0E00E94CA30E4E2EA93E5E9F0E01D
:104484000E94CA30E5E2EA93EFEFF0E00E94CA30FE
:10449400E7E20E94D730E8E20E94D730E9E20E94C6
:1044A400D730EAE20E94D730ECE20E94D730EDE246
:1044B4000E94D730EAE30E94DB30EBE30E94DB305A
:1044C400ECE3EA93E0EFF0E00E94CA30EDE3EA9314
:1044D4000E94EA2C0E94B621E4E1F0E00E94822DC1
:1044E400E5E3EA93E8E3F0E00E94CA30E6E3EA9306
:1044F400E8E7F0E00E94CA30EEE3EA93E8E3F0E094
:104504000E94CA30E0E4EA93EFE0F0E00E94CA308F
:10451400E1E4EA93E0EFF0E00E94CA30E9E1EA93D3
:10452400E9E4F0E00E94CA30E3E9EA93EFE0F0E066
:104534000E94CA300E94E82DE0E2EA93E0E4F0E051
:104544000E94CA30EDE1EA930E94092D0E94B6212F
:10455400EEE1EA930E94EA2C0E94B621EFE10E9468
:10456400CE30E4E4EA93EDE4F0E00E94CA30E5E4FE
:10457400EA93E1E1F0E00E94CA300E94E82DECE108
:104584000E94CE30E4E1F0E00E94822DEBE1EA9358
:10459400E8E1F0E00E94CA300E94DF30EBE1EA93E8
:1045A400E0E1F0E00E94CA300E94DF30E3E4EA93E5
:1045B400E0E8F0E00E94CA30E4E6F0E00E94822DD8
:1045C400E0E9EA93EFE7F0E00E94CA30E6E20E94F5
:1045D400CE300E94DF30E6E2EA93E4E2F0E00E94AB
:1045E400CA30E6E2EA93ECE2F0E00E94CA300E94AC
:1045F400DF30E6E2EA93ECE3F0E00E94CA30E7E55C
:104604000E94D730E5E5EA930E94EA2C0E94B62185
:10461400EEEFEA93EAE5F0E00E94CA30E7E5EA93B8
:104624000E94EA2C0E94B62108950E94E230AE85D1
:10463400AA2362F0AD85BE85A03FE0E0BE0734F456
:10464400AB85BC85AF33E1E0BE070CF05DC00E94D2
:10465400EB2FAE0FBF1FA03FE0E0BE0714F00E9497
:10466400F02F0E94F92FAE0FBF1FA034E1E0BE0768
:1046740014F00E94FE2F49850E94F030E3E0EA9393
:10468400EE85FF850E94CA30E4E00E940B300E9450
:10469400F730E5E00E940B30EA0FFB1F0E94CA309E
:1046A4000E94FD30E7E0EA93EC85FD850E94CA3064
:1046B400E8E00E9418300E94F730E9E00E941830C8
:1046C400EA0FFB1F0E94CA306BDE05BB1BBB2EE149
:1046D4003FE100E010E00E941E3064F050E0451716
:1046E40030F020936500309365005F5FF8CF0F5F73
:1046F4001F4FF1CF64DE0E94C82F0E940431E8E00E
:104704000E94DB300E940B313DC10E94E2300E94C6
:10471400EB2FEA17FB0711F00C94DC230E942330E3
:1047240014F40E942A30E6E1EA93E8EEF0E00E94F5
:10473400CA30E4E00E94DB30E5E0EA93EFE3F1E025
:104744000E94CA30E8E0EA930E94EA2C0E94B62153
:10475400E9E0EA93EFEEF0E00E94CA30E2E0EA9387
:10476400EC85FD850E941031E3E00E9413310E9424
:1047740018310E941D3114DE05BB1BBB2EE13FE145
:104784000B851C850E941E303CF0209365003093FD
:1047940065000F5F1F4FF6CF0E94E1210E94D230C7
:1047A4000E94C82F0E940431E8E00E94DB300E947E
:1047B4000B31E8C00E94F92FEA17FB0751F50E945C
:1047C4003B3014F40E942A300E94F030E3E0EA9374
:1047D400EE85FF85F0700E94CA300E94FD30E7E04C
:1047E4000E9413310E94D22105BB1BBB2EE13FE185
:1047F4000D851E85E985FA85E017F1073CF02093C5
:104804006500309365000F5F1F4FF4CF0E94E121D4
:10481400B9C00E9442300E944930FF93EF930E9436
:104824004D300E944930AF91BF91EA17FB0710F455
:104834000C9466240E94233034F520E030E00E947A
:104844005030E217F307F4F00E9442300E945730D0
:104854000E9450300E9423310E942D31E6E0EA93F9
:10486400AC85BD85A21BB30BFD010E941031E7E0AE
:10487400EA93AC85BD850E9439310E9440312F5F97
:104884003F4FDDCF20C020E030E00E944D30E217E2
:10489400F307CCF00E9442300E9457300E944D3002
:1048A4000E9423310E942D31E6E00E946C300E9468
:1048B400F730E7E00E946C300E9446310E9440319C
:1048C4002F5F3F4FE2CF5EC00E9442300E944930CA
:1048D400FF93EF930E944D300E944930AF91BF91F6
:1048E400EA17FB0710F00C94C4240E943B3034F503
:1048F40020E030E00E947130E217F307F4F00E94E8
:104904004D300E9457300E9471300E944D31AE8567
:10491400BF85A21BB30BFD010E941031E3E0EA93B3
:10492400AE85BF850E9439310E9454310E945A31AC
:104934000E9440312F5F3F4FDDCF24C020E030E0A4
:104944000E944230E217F307ECF00E944D300E94BF
:1049540057300E9442300E944D31F901AE85BF8527
:104964000E94F730E3E0EA93F901AE85BF850E9427
:1049740046310E9454310E945A310E9440312F5FC7
:104984003F4FDECF0E943B352F96089525970E9416
:104994003435EB850E9460310E949130103110F063
:1049A4000C94482500E0E09101030E1710F00C94DC
:1049B40040250E9418310E941D31E0E0EA87AA8553
:1049C400A23010F00C9438250E949D30E252FF4F23
:1049D4002491203011F40C94332527FF39C0E2E0F0
:1049E400EA93FA010E9410310E946C31E2E2E5BBC5
:1049F400E0E0EBBBE7E1E09365001F98F6E1F0939C
:104A04006500E0936500EE81E5BBEF81EBBBEFE170
:104A1400FEE1E0936500F0936500E093650031FFEB
:104A240004C0F0936500E093650026FF10C0F09386
:104A34006500E093650031FF06C0F0936500E093E4
:104A440065004F5F5F4F220F4F5F5F4FEECF1F9A9E
:104A5400220F31FF02C04F5F5F4F4F5F5F4F0C94D7
:104A6400EB24EA85EF5FEA870C94E124ED85FE856B
:104A74003196ED87FE870F5F0C94D524E885F98580
:104A84003296E887F9871F5F0C94D0240C94CE25C6
:104A940023970E943435E9850E94603130910003E8
:104AA40010E0EA851E1710F00C94CE2500E0E0918A
:104AB40001030E1710F00C94CB25E6E0EA93ED8584
:104AC400FE850E941031E7E0EA93ED85FE85F070E3
:104AD4000E94CA30E0E0E887EB85A885AE1710F0A5
:104AE4000C94C3250E94B530203011F40C94BE25DB
:104AF40027FF39C0E2E0EA93FA010E9410310E94D4
:104B04006C31E2E2E5BBE0E0EBBBE7E1E09365009A
:104B14001F98F6E1F0936500E0936500EE81E5BB34
:104B2400EF81EBBBEFE1FEE1E0936500F0936500FC
:104B3400E093650031FF04C0F0936500E0936500E5
:104B440026FF10C0F0936500E093650031FF06C0B6
:104B5400F0936500E09365004F5F5F4F220F4F5F56
:104B64005F4FEECF1F9A220F31FF02C04F5F5F4F9E
:104B74004F5F5F4F0C947625E885EF5FE8870C94D0
:104B84006E25EC85FD853196EC87FD870F5F0C94CF
:104B940059251F5F0C9453250E943B356196089557
:104BA400E1E0E0930B03E8EFFFEFE0932408F093D8
:104BB4002508E491EF3F39F0E0912408F0912508AD
:104BC400049000920B03A0910B03A33019F40E94EC
:104BD400E32102C00E940A1EE3E0E0930203E0E046
:104BE400E0930303E1E0E0930103E0930003EFEEBD
:104BF400F0E0E093FF03F0930004EFE3F1E0E093CF
:104C04000104F0930204E4E1E09306030895A09103
:104C14000B03A33069F40E9471310E9471310E9428
:104C240071310E947131E885EA930E9417230CC008
:104C34000E9471310E9471310E9471310E94713160
:104C4400E885EA930E946D1F1DC0A0910B03A33059
:104C540069F40E9471310E9471310E9471310E9485
:104C64007131E885EA930E9487230CC00E94713158
:104C74000E9471310E9471310E947131E885EA937A
:104C84000E94CE1F29960895A0910B03A33059F4D6
:104C94000E9476310E947631EF81EA93EF81EA93A4
:104CA4000E944A250AC00E9476310E947631EF8123
:104CB400EA93EF81EA930E943A2128960895A091FD
:104CC4000B03A33029F40E947D310E94C82404C040
:104CD4000E947D310E94BC20269608950E94843152
:104CE4001A930A931BB10CB1E0919508F0E0ED59C9
:104CF400F74F0083A0919508AF5FA0939508A23366
:104D040019F4E0E0E093950809911991DBC00E9441
:104D14008431E091FC08A091FB08EA1751F0A091BE
:104D24000108A03029F0A0E00A99A1E0A03009F41C
:104D340001C011C0E091FC08F0E0E956F74FE081B2
:104D4400ECB9A091FC08AF5FA093FC08A43619F459
:104D5400E0E0E093FC08B6C0AA93BA93EA93FA930E
:104D6400EFB7EA931A930A9310919B0000919C0069
:104D7400E12FEC7111F00C942427023021F4E1E0CE
:104D8400E093950A5FC0E091950AE13029F5E0E0EF
:104D9400E093950A0A3229F00E940E2DE05DE01797
:104DA400D1F4E2E0E093950AE0E0E093960A0E94F1
:104DB4008A31E350F74FA2E0A0830E948A31E09346
:104DC400910AF093920A0E948F31E039A1E0FA0728
:104DD40011F40E94923136C0E23071F40093960AC5
:104DE400E3E0E093950A0E949931E039A1E0FA07E3
:104DF40011F40E94923126C0E33021F50E949931CA
:104E0400E039A1E0FA0711F40E9492310330D1F4A1
:104E1400E0E0E093950AA091960AA63529F4E09182
:104E2400FF06E260E093FF06A091960AA33451F4D2
:104E3400689423F8E091910AF091920AE093930A1E
:104E4400F093940A09911991E991EFBFF991E991CD
:104E5400B991A99118951A930E949E310E94A33189
:104E6400D9F30E949E31E350F74F1081AFE8BAE0C6
:104E74000E94432DE039A1E0FA0731F4E0E0F0E0CC
:104E8400E0938F0AF093900AE12F199108950E94FC
:104E94008431E091980BA091970BEA1781F0E0918F
:104EA400FE06E03019F0E89421F808C00E94AA3107
:104EB4000E94B83119F4E0E0E093980B03C0E89441
:104EC40020F821F8E991EFBFF991E991A99118959A
:104ED400E091970BF0E0E956F54FA881A083E091AB
:104EE400970BEF5FE093970B0E94B83119F4E0E061
:104EF400E093970B0C94B92AE0E0E093980BA0910F
:104F0400970BA13020F00E94AA31689421F80895EB
:104F1400AA93BA93EA93EFB7EA93E0E0E093980B8D
:104F24000E940E2DEF5FE093FE06E991EFBFE99139
:104F3400B991A99118952A970E94343520E00E94CE
:104F44009E310E94A33121F0A091990BA23008F068
:104F54002FC023FE0AC0E091930AF091940AE093D3
:104F64008F0AF093900AE89423F875DF1E2F12300D
:104F740029F4E1E0E093990BE0E017C0A091990BCC
:104F8400A130A9F40E94BD311083133039F4E2E05A
:104F9400E093990B0E94BD31A0E0A083A0919A0BED
:104FA400AC3328F4E0919A0BEF5FE0939A0BC7CFF0
:104FB400A091990BA23011F00C94942921E0E09176
:104FC4009B0BE33471F4E0919C0BE7703E2F30307F
:104FD40019F40E943E1A04C00E94C3310E94721A3E
:104FE4009DC1E43471F4E0919C0BE7703E2F3030A6
:104FF40019F40E940C1D04C00E94C3310E941F1D9D
:105004008DC1E73499F5E0919E0BE73469F4A091E2
:10501400FC06A53149F0E0919C0BE053AE2FE091E2
:105024009D0BE055EA1709F020C0E0919C0BE0537A
:10503400A8E0B0E00E949F330E94EA2C0E94EA2C70
:10504400EFEEF0E00E94DD310E94F42C0E94EA2C85
:105054000E94EA2C0E94171AE6EEF3E20E94052D44
:105064000E940E2DF0E00E94A72D58C1E93431F4BE
:10507400E0919C0BE370E093FC0350C1E134E1F454
:10508400E0919C0BEF70E0930203E0919D0BEF70B5
:10509400E0930303E0919E0BEF70E0930403E0912F
:1050A4000303A0910203EA1731F4A0910303EFE094
:1050B400EA27E093020332C1EC3439F4E0919C0B0B
:1050C400E170EA930E94331229C1E43511F00C9483
:1050D400D928A0910503A03041F4A0919C0BA133E1
:1050E40020F0A0919C0BAA3308F01EC0E0919D0B08
:1050F400E153A8E9B0E00E94E231E0919C0BE15356
:105104000E2F0E94EC310E9471330E942C2F0E94BA
:10511400EC3132960E947133FA93EA93EAE3F0E0B9
:105124000E94F5310E94FB31A0910503A13041F4A6
:10513400A0919C0BA13320F0A0919C0BA43308F008
:1051440014C0E0919C0BE153AEE4B1E20E94E23161
:10515400E0919D0BE153A2E4B1E20E940132EAE343
:10516400F0E00E940C320E94FB31A0910503A230B2
:1051740041F4A0919C0BA13320F0A0919C0BA4338B
:1051840008F014C0E0919C0BE153A8E5B1E20E9441
:10519400E231E0919D0BE153A4E5B1E20E940132BA
:1051A400EAE9F0E00E940C320E94FB31B7C0E5341A
:1051B400A1F4E0919C0BE053E0939F06E0919D0BDA
:1051C400E153E093A006E0919E0BE13311F4E1E09A
:1051D40001C0E2E0E0932608A1C0E63459F4A091AE
:1051E4009C0BA03320F0A0919C0BA33308F001C0CA
:1051F40095C002C0E63521F4E0E0E0939C0B8EC03C
:10520400E83511F00C948A29E0910503E03031F47B
:10521400E0912608E0930003E1E004C0E1E0E093BC
:105224000003E2E0E093010322FC02C00E943C126E
:10523400689422F8A091A006E4E1EA9FF001A0910D
:105244000103EA9FF001EE5FF0E0EA87FB870E942A
:10525400AE2EF0E0E887F987E0910103A4E1EA9F2C
:10526400F001F0E0EE83FF8331E00E941132E03080
:1052740011F40C948929A0919F06A43120F4A091E3
:10528400A006A33008F041C0E0919F06A3E0EA9F86
:10529400F001E95DF74FDF01E091A006F0E0AE0F09
:1052A400BF1F0E941132EC93E0919F060E94982E3A
:1052B400DF01E0910003F0E00E94D732EC87FD8724
:1052C400E0910503E03029F0EC85FD853A96EC8702
:1052D400FD870E9417320E9417320E941732EC8514
:1052E400FD850E94F42C0E941732EC85FD850E94F6
:1052F400A32D0E941132EA93E0E0EA930E94B819C8
:10530400E0919F06EF5FE0939F063F5FAECF06C03C
:10531400E93521F40E94BE16E89422F8E0E0E09317
:10532400990BE22F0E943B3560960895A0E020FC83
:10533400A1E0A03029F4E091FF06E270E23009F028
:1053440010C00E941C32E05DEA93C2DDE6E5EA93F8
:10535400BFDDE2E30E942432ED7FE093FF06689410
:1053640020F8A0E020FCA1E0A03029F4E091FF06A1
:10537400E370E13009F020C00E941C32E05DEA9342
:10538400A7DDE4E5EA93A4DDE091FC06EA93A0DD61
:10539400E0912008E295EF70EA9326D0EA9398DD35
:1053A400E0912008EF70EA931FD00E942432EE7F30
:1053B400E093FF06689420F8A0E020FCA1E0A1306F
:1053C40049F4A0E021FCA1E0A03021F4A091FE0664
:1053D400A03009F001C090DDE091FE06E03019F044
:1053E400E150E093FE060895A881AA3020F4E881F4
:1053F400E05D0C94B92AA881AA3020F0E881E95C28
:105404000C94B92AE8E50C94B92A0E942E320E9421
:1054140033320E94DD310E9436320E942E320E94C5
:105424007D2DE4E1F0E00E94DD310E943632E2EDB0
:10543400F0E0FA93EA930E9433320E94DD310E9435
:105444003632E2EDF0E0FA93EA930E947D2DE4E136
:10545400F0E00E94DD310E943632E4E1F0E0FA939C
:10546400EA930E942E32E8ECF0E0FA93EA93ECE33C
:10547400F0E00E943C320E9433320E94DD310E94EF
:105484004232E2EDF0E00E94DD310E94DD310E9403
:105494004232EFE0E0930303E2E0E0930003E093A1
:1054A4000103E5E5F0E0FA93EA93EEE1F0E00E940F
:1054B400A32DECEEF3E20E94052D0E94FA2CE0E00D
:1054C400E09303030895EEE5F1E2FA93EA93EAEB3D
:1054D400EA93EAEFF0E0FA93EA93E4E0EA93E6E28F
:1054E400EA93EEE0EA930E944626E6EFF1E2FA93AD
:1054F400EA93EAEAEA93E7E0F1E0FA93EA93E8E070
:10550400EA93E2E3EA93E1E0EA930E9446260895EF
:10551400E991F991A991B991CD0161916D936623B6
:10552400E1F7FC010895E991F991A991B991CD01AF
:1055340005900D920020E1F7FC010895A991B9911D
:10554400EE27FF276D91662311F03196FBCF089566
:10555400AA27BB27E991F9910590002011F0119633
:10556400FBCFFD0108955D9BFECFE881ECB9219648
:1055740008951A930A93AC81BD810E9467333097D2
:10558400C1F0AA81BB810E9467338F01309749F033
:105594000230E0E01E0760F0F80131978F01ED93CF
:1055A400FC93AC81BD810E94432D3197AE81A083D1
:1055B40003C0EE81EA93D7DF198108812796089505
:1055C4002C970E94343510E0E88DF98D3196E88FE0
:1055D400F98F3197E4912E2FE03011F40C949E2C26
:1055E400E12FE03039F4253211F411E002C00E94B9
:1055F4004732A1C1E130C1F4253219F40E94473287
:1056040099C112E0E0E0E98B00E02D3211F401E0F1
:1056140092C12B3219F4EBE2E98B8DC1203219F4DB
:10562400E0E2E98B88C102C0E23039F450E013E0D3
:10563400203311F400687FC102C0E330A1F42033A9
:1056440010F02A3308F009C0A52FEAE0EA9FF00120
:105654005E2FE22FE0535E0F6EC140E02E3211F454
:1056640014E069C110C0E430A1F4203310F02A33EF
:1056740008F009C0A42FEAE0EA9FF0014E2FE22FC0
:10568400E0534E0F58C12C3619F4026015E053C193
:1056940004C0E53011F00C949D2CE22FE33649F45C
:1056A4000E945232EE89FF89A481AA930E94583243
:1056B40041C1E33741F40E9452320E9462320E9497
:1056C400A02A1E2F0AC0E037A1F40E9452320E9481
:1056D40062320E94AA2A1E2F08600F77403011F010
:1056E400411708F001C0142F40E0E0E0E88B30E0FF
:1056F40078C0E43611F0E93611F4046002C0E537ED
:10570400A1F4EAE0E88B01FF08C0E0E0FAEC6AE902
:105714007BE30E94642D1AE023C0E0E1F7E260E03D
:1057240070E00E94642D15E01BC0E83511F4086098
:1057340004C0E83711F00C949C2CE0E1E88B01FFE5
:1057440008C0E0E0F0E060E070E10E94642D18E041
:1057540007C0E0E0F0E160E070E00E94642D14E036
:10576400403011F00F7701C041E001FF08C00E94F2
:105774005232AE89BF8914960E946B3315C002FF62
:105784000AC00E945232AE89BF8914960E946733C0
:105794000E94A43209C00E945232AE89BF89149675
:1057A4000E94673366277727EC87FD876E877F879C
:1057B40002FF16C0AF85AA2362F4EC85FD856E85D1
:1057C4007F850E948E32EC87FD876E877F87EDE2AE
:1057D400E98BE989E03019F01F5F4F5F01C00B7F4F
:1057E400342F00FD14C0151710F4351708F00FC03E
:1057F40007FF08C002FF04C00B7F2989115001C0B4
:1058040020E301C020E20E9447325150ECCF14172C
:10581400B0F4006102FF0AC00B7FE989EA930E9499
:105824005832503009F0515011504150E0E3EA939E
:105834000E945832503009F051504150E8CF312F76
:10584400E889E030D1F43030B9F003FF08C0EE81CC
:10585400FF813196EE83FF833197E49105C0AE81D9
:10586400BF81ED91AE83BF83EA930E9458325030DA
:1058740009F051503150E7CF53C00E946C320E945E
:1058840007332E2F2A3030F003FF02C0295C01C0F9
:10589400295A01C0205D04FD23C0213350F40E9425
:1058A400692DA130E0E0BE07E0E08E07E0E09E074E
:1058B40009F40BC0431740F4531710F000FF01C064
:1058C40014C020E207FF0CC020E3006102FF08C0FF
:1058D4000B7FE989EA930E945832503009F0515005
:1058E4000E944732503009F0515031500E946C32BE
:1058F4000E944233EC87FD876E877F87E8890E9488
:10590400692DFF27662777270E9407330E94642D9D
:10591400E885F9856A857B850E942C3509F0ADCF31
:1059240000FF08C0503031F05150E0E2EA930E9489
:105934005832F8CF10E048CE0E943B356A9608955D
:10594400FF92F82E22971A930A93DE010E94813265
:105954008D01DE0116960E9481320E946733EA832C
:10596400FB83DE0114960E9481320E946733FA930E
:10597400EA931A930A930E94572E0E94EA2C20DE7F
:10598400AA81BB81E0E0EC93198108812496FF9001
:105994000895A991B991EE27002460E8E894162EA1
:1059A400169407941E2A1EF0A015B10518F0A0192C
:1059B400B109E62BB7FBAA0FBB1F669580F70895C4
:1059C400E991F99130971AF4E095F095319608959C
:1059D400E0E0F0E0FA93EA930895E091FF03F09198
:1059E40000040895FA93EA93EFE0EA930C940926ED
:1059F400E1E0E0930003E09301030895E6E0F0E0C2
:105A0400FA93EA930895FA93EA930C94FB16E7E069
:105A1400F0E0FA93EA930895A8E0B0E00E948B3393
:105A24000895E093620088EC90E00197F1F70895FF
:105A3400E093610088EC90E00197F1F70895E0911C
:105A44008F06F09190060895E0918B06F0918C06F4
:105A54000895AE0FBF1FE3E0F0E00E940233089503
:105A6400FA93EA931A930A930C947A12FA93EA93A8
:105A74003A932A930C947A12A0918706B0918806DF
:105A84000895ED91FD913196FE93EE930895A091C2
:105A94009306B09194060895A0919506B091960648
:105AA4000895E0937906F0937A060895A0E0B0E0B3
:105AB4000E94873308950E948033EA1BFB0B0E94E7
:105AC400A4320895E887F9876A877B870895A885B3
:105AD400B9858A859B850895A2E0B0E00E9487334A
:105AE4000895A4E0B0E00E9487330895A6E0B0E0F2
:105AF4000E9487330895E2E3F0E0FA93EA9308956D
:105B0400FA93EA930C947532A0918106B0918206BF
:105B14000895E0EAF0E0FA93EA930895EA930E9484
:105B24000F1AE1E0E09300030895EAE0EA930E948B
:105B34008B16E0919306F091940608950E94973392
:105B4400DACFFA93EA930C94321AFA93EA930C9408
:105B5400DB16E8E1F0E0FA93EA93E8E2F0E042CF02
:105B6400E7EDF0E0FA93EA93D4CFE2E0E0930003A8
:105B7400E9E6F0E0FA93EA930895EAE0EA930E94F2
:105B84008B16E0919506F091960608950A921A9262
:105B9400FA926A937A938A939A93AA93BA93EA931A
:105BA400FA93EFB7EA930895ACE01A9FF001E45F2B
:105BB400FC4FE0810895ACE01A9FF001EB5EFC4FCE
:105BC40008951A93E1E0EA930C949F1AEAE0F0E056
:105BD40097CFE093E206F093E3060895A981BA8192
:105BE400EE27A10FBE1FEC910895FE01FA93EA93EC
:105BF40008950E94753384E00E94A22C2896F5CF64
:105C0400F801AA81BB81EA0FFB1FE4910895E0919A
:105C1400E506A8EEB6E0F0E0EE0FFF1F0895E09170
:105C2400E406A8EEB6E0F0E0EE0FFF1FEA0FFB1F5C
:105C34000895E981ACE0EA9FF0010895EF73A9E2C9
:105C4400EA9FF001E757FB4F0895EF73ABE0EA9F3B
:105C5400F001EB5FFB4F0895ACE01A9FF001E15FA8
:105C6400FC4F0895ACE01A9FF001E35FFC4FDF01A5
:105C74000E9467330895ACE01A9FF001E35FFC4F84
:105C8400608171811A9FF001EF5EFC4FE081DB01BE
:105C9400F0E00895A083ACE01A9FF0010895ACE011
:105CA4001A9FF001EA5EFC4F0895FE013696FA93BE
:105CB400EA930895FA93EA930C948A2AA9E20A9F34
:105CC400F001E757FB4FE081E0300895A9E20A9F15
:105CD400F001E757FB4FFA93EA93FE013896EACFB7
:105CE400ABE00A9FF001EB5FFB4FE081E0300895E9
:105CF400E091E206F091E3060895A2EEB6E0ED919C
:105D0400FD913296FE93EE930895E081F0E0E60F64
:105D1400F71F0895E0938906F0938A060895E0E05A
:105D2400F0E0E0938706F09388060895F0E0ACE095
:105D3400B0E00E94D73208951A930A933A932A93B3
:105D44000895E0910103F0E00895FA93EA93ED8158
:105D5400EA93ED81EA930895E0910003ACE0EA9FB1
:105D6400F0010895F0E0EA0FFB1F0895E0930703A4
:105D7400F093080308951A93E1E0E0930103E0939C
:105D8400000310E00895DF010E946733DF01EB8117
:105D9400FC810895DF010E946733DF01E981FA8104
:105DA4000895EF81F885EA1BFB0B0895FE01EB5B78
:105DB400FF4FE081ACE0EA9FF001EA5EFC4FE08136
:105DC4000895FE01EB5BFF4FE081ACE0EA9FF00138
:105DD4000895ECE8F0E00E9471330895DE01A05CC0
:105DE400BF4FED93FC930895FE01E85BFF4F0190D4
:105DF400F081E02D0895FA01E00FF11FFA93EA9380
:105E04000895E0E0EA930C9427261A930A93FE017E
:105E1400EC5BFF4F0190F081E02DE20FF31F08953A
:105E2400FA93EA93E8CFE0DFE20FF31FFA93EA93E1
:105E3400E8CFE0E0EA930C940926FA93EA933A93C4
:105E44002A930895E5E0F0E0FA93EA93CDDFFA931C
:105E5400EA93EFCFFA93EA935A934A930895DE01B3
:105E6400AC5BBF4FAC910895DA01F0E00895DF0117
:105E7400FE01EE5BFF4F0190F081E02DAE17BF07EE
:105E84000895FE01EE5BFF4F0190F081E02D08952F
:105E9400E2E0F0E00E9402330895A0DFDE01AF5B90
:105EA400BF4FAC91AA230895ECE0EA9FF001A091C2
:105EB4000003EA9FF0010895AE1BBF0BE9CFECADE0
:105EC400F0E0E00FF11F08953196FA93EA93D9DFD9
:105ED400E20FF31F319635CEFA93EA93D2DFE20F45
:105EE400F31F2FCEEFADF0E0DE011696AE0FBF1F0D
:105EF400EC910895EA93EBADEA930E94B819EFADE3
:105F0400EF5FEFAF0895F0E0DE011696AE0FBF1F0E
:105F1400AC9108950E94D732E20FF31FDF01B1DF85
:105F2400EE0FFF1FEA0FFB1F08950E94D7320E9455
:105F3400A4320E9416340895E98DFA8DE21BF30B06
:105F4400FA93EA930895FA93EA93F901AD8DBE8D1D
:105F5400EA0FFB1FFA93EA930895FA93EA93EA8D02
:105F6400EA930C942726EBE1E0936500E4E6F0E085
:105F7400C7CDFA93EA930C94E61DEA93E1E0F0E0CE
:105F8400F8CFE3E0EA93E0E3F0E1F3CFE4E0EA936F
:105F94001FCDEA93E7E0F7E0ECCF0E94E61DE1E5D0
:105FA400EA93EFEEF0E0E5CF0E94E61DE3E5EA9325
:105FB400EFE3F1E0DECF0E943435EE81AEEDB0E2E6
:105FC400F0E0EE0FFF1FEA0FFB1F0E9471338F01F9
:105FD4000895E985FA85AD85BE850895AD85BE85AC
:105FE400EFEEF0E0EA1BFB0BE987FA870895EF81F7
:105FF400F885AB85BC850895AB85BC85EFE3F1E0FE
:10600400EA1BFB0BEF83F8870895EA93EE85FF857F
:10601400B0CFEA93EA85FB85AE85BF850895EA0F84
:10602400FB1FA7CFEA93EC85FD85A3CFEA93E88510
:10603400F985AC85BD850895EF81F885E017F107F2
:106044000895EB85FC85AF81B885AE17BF07089529
:106054000D851E85ED85FE85E987FA870D871E87E8
:106064000B851C85EB85FC85EF83F8870B871C87E4
:106074000895ED85FE85A985BA85AE17BF070895F5
:10608400AD85BE85E985FA85EA1BFB0B0895FA9375
:10609400EA930C94E22CAB85BC8583CEAF81B885A2
:1060A400EB85FC85EA1BFB0B0895D9010E94D732CE
:1060B4000F010895D0010E940233AF01E0E2EA9398
:1060C400FA01AE85BF85ABCFE2E2EA931A930A9355
:1060D4000C94E61DEA93F901AC85BD850895A98564
:1060E400BA85ED85FE85EA1BFB0B0895D0010E945D
:1060F4000233AF01E0E2EA930895E1E2EA93FA01A0
:10610400AC85BD858CCFAEEDB0E2F0E0EE0FFF1FA5
:10611400EA0FFB1F0E947133EE83FF830895EC8521
:10612400F0E0EE0FFF1F0E949632E887F987309166
:10613400000310E00895EA85F0E00E949832DF0140
:10614400E32FF0E00E94D732AF85B889EA0FFB1F36
:10615400AF01EA85A885B98505CEE0E2EA935A93B2
:106164004A930C94E61DE885F0E00E949832DF0122
:10617400E32FF0E00E94D732AE85B0E0EA0FFB1FB8
:10618400AF01EF85F88924913196EF87F88B089554
:10619400FA93EA930C94B621EA93E4E0F0E0F8CFA2
:1061A400E6E1EA93E8ECF0E0F3CFEA93E2E0F0E032
:1061B400EFCFEA93E1E0F0E0EBCFE8E2F0E0A0CC4F
:1061C4000E943435EE81AEEFB0E2F0E0EE0FFF1F37
:1061D400EA0FFB1F0E9471338F010895E2E0EA93F6
:1061E400EE85FF850E949F32D3CFAE0FBF1FFD0106
:1061F4000E949F32CDCFE6E0EA93EC85FD850E94B4
:106204009F32C6CF0E94B621E5E0EA93EFEEF0E0BC
:10621400BFCFE9E0EA93EFE3F1E0BACF0E949F3207
:10622400B7CFEA93EC85FD85F070B2CFE6E0EA9350
:10623400EE85FF85F3CFE7E0EA93EE85FF85F07006
:10624400A7CFD0010E940233AF01E2E0EA93FA0142
:10625400AE85BF85CACFE3E0EA93FA01AE85BF8578
:10626400AE0FBF1FEFEFF0E0EA23FB2391CFA21B99
:10627400B30BEFEFF0E0EA23FB238ACFE2E2EA93E9
:106284001A930A930C94B621AE0FBF1FEFEFF0E000
:10629400EA23FB237DCFD0010E940233AF01E2E069
:1062A400EA930895E6E0EA93FA01AC85BD859DCFB3
:1062B400E7E0EA93FA01AC85BD85E6CFAEEFB0E244
:1062C400F0E0EE0FFF1FEA0FFB1F0E947133EE8315
:1062D400FF830895E3E0EA93FA01F07059CFEF8168
:1062E400F885FA93EA930895EE81FF81FA93EA938D
:1062F400EF81EA930895EC81FD81FA93EA93EC81AE
:10630400FD8123CDAA93EA93FA93EFB7EA93089514
:10631400E0918D0AF0918E0A0895ADE8BAE0B1CB10
:10632400E0E0F0E0E0938D0AF0938E0A0895F0DF48
:10633400E350F74F0083F1CFE0918F0AF091900A78
:106344000895A0918D0AB0918E0AEA17FB0708956B
:10635400E091980BF0E0E956F54FE081E0939C0062
:10636400E091980BEF5FE093980B0895F0E0E03034
:10637400A1E0FA070895E0919A0BF0E0E556F44F96
:106384000895E32FE150A8E9B0E0F0E0EE0FFF1F1D
:10639400EA0FFB1F0E947133FA93EA93E32FA8E9F3
:1063A400B0E0F0E0EE0FFF1FEA0FFB1F0E94713315
:1063B400FA93EA930895FA93EA93E4E1F0E00895F6
:1063C400F0E0EE0FFF1FEA0FFB1F0E9471333396BC
:1063D400AF010895E02FAEE1B1E2F0E00E949A32FD
:1063E400EA0FFB1F0895FA93EA93E0919E0BEA9358
:1063F400EFCAEFE9FBE0FA93EA930C946C17F0E030
:10640400EE0FFF1FEA0FFB1F0E9471333396EE87D6
:10641400FF8720CDFA93EA93EAE4F0E0E4CFE32F98
:10642400F0E0E556F44FE0810895EC85FD85FA939C
:10643400EA930895E0E0E093970BE2E0EA930E9488
:106444006A27EACAEA930E946A27E3E0EA930E9471
:106454006A27E091FF060895EAE0F0E0FA93EA93F0
:106464000895EAE0F0E0A7CFFA93EA93ECE0EA9328
:106474000C94591DFA93EA93ECE0EA930C940926E0
:10648400FA93EA93E8E2F0E0F5CF2A93ED89FE89E6
:10649400FA93EA93FE017596FA93EA930C94BB2A55
:1064A400EE89FF893497EE8BFF8B0895ED89FE8981
:1064B400FA93EA93FE017596FA93EA930C94BB2A35
:1064C400AE89BF8914960E946733EE83FF83FA93E3
:1064D400EA930895E885F9856A857B85AC85BD8551
:1064E4008E859F850895E991F991309639F080EA77
:1064F4009FE00197F1F7A8953197C9F70895002413
:10650400AF0DB01D0895EA1BFB0B680B790B0895C2
:10651400F195E195F0400895F09560957095E195B9
:10652400FF4F6F4F7F4F0895EE0FFF1FEE0FFF1FBA
:10653400EE0FFF1FEE0FFF1F0895EF2FFF27E7FD5C
:10654400FFEF08956F2F660F660B762F0895EA17F5
:10655400FB07E1E00CF0EE270895FA9FF02DEB9F86
:10656400F00DEA9FE02DF10D08957A9F702D6B9F39
:10657400700DF89F700DE99F700D6A9F602D710D6D
:10658400FB9F600D711DE89F600D711D8827FA9FA8
:10659400F02D610D781FEB9FF00D611D781FEA9FB0
:1065A400E02DF10D681F781F08956ED0D6DF0EF42C
:1065B400AFDF089577D0D9DF0EF4AEDF089500245D
:1065C40098E0AA0F001C0E1A10F40E0E01C0A16070
:1065D4009A95B9F7EA2FA02D08950024112490E18B
:1065E400AA0FBB1F001C111C0E1A1F0A18F40E0E52
:1065F4001F1E01C0A1609A9599F7FD01D00108956D
:1066040043D0EBDF0EF484DF08953F934F935F9301
:10661400002411244427552730E2AA0FBB1F881FEA
:10662400991F001C111C441F551F0E1A1F0A460BEC
:10663400570B28F40E0E1F1E461F571F01C0A160E2
:106644003A9559F7FD01BC01D001CA015F914F9100
:106654003F91089527D0D9DF0EF45EDF0895AFDFB0
:10666400EA2F0895E894B7FF04C0A095B095119659
:106674006894F7FD4DDFB1DFFD010EF449DF0895A5
:10668400C4DFFD01BC010895E894F7FF02C040DFB8
:106694006894B7FF06C0A095B095119600F80394CE
:1066A40000FA0895E89477FF02C036DF689497FFF4
:1066B4000BC00024A095B095809590951196801DEF
:1066C400901D00F8039400FA0895ED91FC91119740
:1066D4000895ED91FD916D917C9113970895059026
:1066E400F491E02D08957A936A93FA93EA930895C6
:1066F400182E862F612D192E972F712D1B2EBF2F2B
:10670400F12D1A2EAE2FE12D0895119602D0FE2FF1
:106714001197E199FECFFF93FFB7F894AEBBBFBBCF
:10672400E09AEDB3FFBFFF91089507D01196EF9360
:10673400EF2F03D0EF9111970895E19B02C0A89524
:10674400FCCF9FB7F894AEBBBFBBE09A8DB3E817FC
:1067540019F0EDBBE29AE19A9FBF0895552342F4E4
:10676400503811F4E0FF04C03196691F791F6BF0B3
:1067740050E8572711F45F93C8C05F3F31F0660FAC
:10678400000C57956795752F08955F9300200AF0C4
:10679400C8C0C1C050E8192E1522880F991F95272B
:1067A400550F879550E8072E0522660F771F75272A
:1067B400550F67950895689401C0E8945F93F2DFDC
:1067C400703818F07F3F08F4A0C056E1571BAAF4B4
:1067D400519558300EF4593030F0EFEFFFEF6FEF72
:1067E4007FE777F91AC077275523B9F0EE0FFF1F1B
:1067F400661F771F5A95D1F710C07727583028F0B5
:10680400EF2FF62F672F5850F9CF552331F0769597
:106814006795F795E7955A95D1F700200AF47CDE41
:106824005F910895689401C0E89430976040704087
:10683400B1F0002426F0772312F400946DDE172EB5
:106844007EE1112032F07A95EE0FFF1F661F111CB6
:10685400F9CFEF2FF62F612D5F938ADF5F910895B3
:106864004F93AF01FD01DA01AB01BC01CA01402D18
:10687400012C142E4F910895EA0FFB1F681F0895F1
:10688400E095F0956095EF5FFF4F6F4F08955F932C
:1068940081DF903849F150E81526703821F1572FDF
:1068A400591B13F112F4DCDFFACF583118F0AA2780
:1068B400BB278827583028F0AB2FB82F882758508B
:1068C400F9CF552329F08695B795A7955A95D9F709
:1068D400502D512562F0D0DF38F46795F795E79590
:1068E400739513F41EC0BCDF43DF5F910895EA1B68
:1068F400FB0B680B51F010F40094C2DF6623A2F383
:10690400EE0FFF1F661F7A95CBF7EE27FF2766274A
:1069140077275F910895EFEFFFEF6FE77FEF5F91C8
:106924000895EFEFFFEF6FE77FE75F9108955F93BF
:1069340031DF703851F3903841F301240894791F02
:1069440023F41CF300203AF3ECCF0F921F932F9300
:106954003F934F93112722279927689FA0018F9F68
:10696400302D410D591F6B9F300D411D591F8E9FB6
:1069740027D0BF9F25D06A9F23D0BE9F1DD0AF9F35
:106984001BD0AE9F110D291F391F491F591FE32F1B
:10699400F42F652F522F4F913F912F911F910F90FC
:1069A40066232AF0550FEE1FFF1F661F02C0739562
:1069B4004BF2D4DE5F910895100D211D391F02C0E2
:1069C400200D311D491F591F08955F93E3DE703870
:1069D40021F411200AF49FCFA4CF903809F495CF65
:1069E40001240894970B1BF4D4F30020F3CF792FE0
:1069F4001F932F933F934F9311241127222733275B
:106A04004427552790E2AE17BF078607410730F0A9
:106A1400AE1BBF0B860B410B089401C08894551F15
:106A2400221F331F111CAA1FBB1F881F441F9A95C6
:106A340051F7F901612D4F913F912F911F916623D9
:106A440032F0550FEE1FFF1F661F7A9543F286DE64
:106A54005F910895309760407040089500240A16AD
:106A64000B0608955A934A933A932A931A930A93D6
:106A740008955D814C813B812A81198108810895A3
:00000001FF
